 isobsolete001

 Timestamp is 7505d23a (reproducible build file hash)

 Preferred load address is 0000000180000000

 Start         Length     Name                   Class
 0001:00000000 000048b0H .text$mn                CODE
 0001:000048b0 00000036H .text$mn$00             CODE
 0001:000048e6 00000092H .text$x                 CODE
 0002:00000000 000001c8H .idata$5                DATA
 0002:000001c8 00000038H .00cfg                  DATA
 0002:00000200 00000008H .CRT$XCA                DATA
 0002:00000208 00000008H .CRT$XCZ                DATA
 0002:00000210 00000008H .CRT$XIA                DATA
 0002:00000218 00000008H .CRT$XIC                DATA
 0002:00000220 00000008H .CRT$XIZ                DATA
 0002:00000228 00000008H .CRT$XLA                DATA
 0002:00000230 00000008H .CRT$XLZ                DATA
 0002:00000238 00000008H .CRT$XPA                DATA
 0002:00000240 00000008H .CRT$XPZ                DATA
 0002:00000248 00000008H .CRT$XTA                DATA
 0002:00000250 00000010H .CRT$XTZ                DATA
 0002:00000258 00000000H .gehcont$y              DATA
 0002:00000258 00000000H .gfids$y                DATA
 0002:00000260 00002e20H .rdata                  DATA
 0002:00003080 00000000H .rdata$CastGuardVftablesA DATA
 0002:00003080 00000000H .rdata$CastGuardVftablesC DATA
 0002:00003080 00000028H .rdata$T                DATA
 0002:000030a8 000000bcH .rdata$voltmd           DATA
 0002:00003164 0000031cH .rdata$zzzdbg           DATA
 0002:00003480 00000008H .rtc$IAA                DATA
 0002:00003488 00000008H .rtc$IZZ                DATA
 0002:00003490 00000008H .rtc$TAA                DATA
 0002:00003498 00000008H .rtc$TZZ                DATA
 0002:000034a0 00000004H .tls                    DATA
 0002:000034a4 00000004H .tls$                   DATA
 0002:000034a8 00000008H .tls$ZZZ                DATA
 0002:000034b0 000003c0H .xdata                  DATA
 0002:00003870 00000368H .edata                  DATA
 0002:00003bd8 0000008cH .idata$2                DATA
 0002:00003c64 00000014H .idata$3                DATA
 0002:00003c78 000001c8H .idata$4                DATA
 0002:00003e40 00000486H .idata$6                DATA
 0003:00000000 00000080H .data                   DATA
 0003:00000080 0001b238H .bss                    DATA
 0004:00000000 000003fcH .pdata                  DATA

  Address         Publics by Value              Rva+Base               Lib:Object

 0000:00000000       __AbsoluteZero             0000000000000000     <absolute>
 0000:00000000       ___safe_se_handler_count   0000000000000000     <absolute>
 0000:00000000       ___safe_se_handler_table   0000000000000000     <absolute>
 0000:00000000       __arm64x_extra_rfe_table   0000000000000000     <absolute>
 0000:00000000       __arm64x_extra_rfe_table_size 0000000000000000     <absolute>
 0000:00000000       __arm64x_native_entrypoint 0000000000000000     <absolute>
 0000:00000000       __arm64x_redirection_metadata 0000000000000000     <absolute>
 0000:00000000       __arm64x_redirection_metadata_count 0000000000000000     <absolute>
 0000:00000000       __dynamic_value_reloc_table 0000000000000000     <absolute>
 0000:00000000       __enclave_config           0000000000000000     <absolute>
 0000:00000000       __guard_check_icall_a64n_fptr 0000000000000000     <absolute>
 0000:00000000       __guard_eh_cont_count      0000000000000000     <absolute>
 0000:00000000       __guard_eh_cont_table      0000000000000000     <absolute>
 0000:00000000       __guard_fids_count         0000000000000000     <absolute>
 0000:00000000       __guard_fids_table         0000000000000000     <absolute>
 0000:00000000       __guard_iat_count          0000000000000000     <absolute>
 0000:00000000       __guard_iat_table          0000000000000000     <absolute>
 0000:00000000       __guard_longjmp_count      0000000000000000     <absolute>
 0000:00000000       __guard_longjmp_table      0000000000000000     <absolute>
 0000:00000000       __hybrid_auxiliary_iat     0000000000000000     <absolute>
 0000:00000000       __hybrid_auxiliary_iat_copy 0000000000000000     <absolute>
 0000:00000000       __hybrid_code_map          0000000000000000     <absolute>
 0000:00000000       __hybrid_code_map_count    0000000000000000     <absolute>
 0000:00000000       __x64_code_ranges_to_entry_points 0000000000000000     <absolute>
 0000:00000000       __x64_code_ranges_to_entry_points_count 0000000000000000     <absolute>
 0000:00000100       __guard_flags              0000000000000100     <absolute>
 0000:00000000       __ImageBase                0000000180000000     <linker-defined>
 0001:00000000       ?NewObject@JNIEnv_@@QEAAPEAV_jobject@@PEAV_jclass@@PEAU_jmethodID@@ZZ 0000000180001000 f i libisobsolete001.obj
 0001:00000028       ?TranslateError@@YAPEBDW4jvmtiError@@@Z 0000000180001028 f   libisobsolete001.obj
 0001:000002e0       ?nsk_jni_check_exception@@YAHPEAUJNIEnv_@@QEBDH@Z 00000001800012e0 f   libisobsolete001.obj
 0001:00000424       ?nsk_jni_lverify@@YAHHPEAUJNIEnv_@@HQEBDH1ZZ 0000000180001424 f   libisobsolete001.obj
 0001:000004c4       Agent_Initialize           00000001800014c4 f   libisobsolete001.obj
 0001:000006a0       Agent_OnAttach             00000001800016a0 f   libisobsolete001.obj
 0001:000006a0       Agent_OnLoad               00000001800016a0 f   libisobsolete001.obj
 0001:000006a8       Java_nsk_jvmti_unit_FollowReferences_FollowRefObjects_addRefToVerify 00000001800016a8 f   libisobsolete001.obj
 0001:00000880       Java_nsk_jvmti_unit_FollowReferences_FollowRefObjects_getTag 0000000180001880 f   libisobsolete001.obj
 0001:00000940       Java_nsk_jvmti_unit_FollowReferences_FollowRefObjects_resetRefsToVerify 0000000180001940 f   libisobsolete001.obj
 0001:00000948       Java_nsk_jvmti_unit_FollowReferences_FollowRefObjects_resetTags 0000000180001948 f   libisobsolete001.obj
 0001:0000098c       Java_nsk_jvmti_unit_FollowReferences_FollowRefObjects_setTag 000000018000198c f   libisobsolete001.obj
 0001:00000be4       Java_nsk_share_jvmti_ArgumentHandler_getAgentOptionsString 0000000180001be4 f   libisobsolete001.obj
 0001:00000c94       Java_nsk_share_jvmti_DebugeeClass_checkStatus 0000000180001c94 f   libisobsolete001.obj
 0001:00000d1c       Java_nsk_share_jvmti_DebugeeClass_resetAgentData 0000000180001d1c f   libisobsolete001.obj
 0001:00000d7c       Java_nsk_share_jvmti_RedefineAgent_agentStatus 0000000180001d7c f   libisobsolete001.obj
 0001:00000d88       Java_nsk_share_jvmti_RedefineAgent_isRedefined 0000000180001d88 f   libisobsolete001.obj
 0001:00000d94       Java_nsk_share_jvmti_RedefineAgent_redefineAttempted 0000000180001d94 f   libisobsolete001.obj
 0001:00000da0       MA_checkStatus             0000000180001da0 f   libisobsolete001.obj
 0001:00000e44       __local_stdio_printf_options 0000000180001e44 f i libisobsolete001.obj
 0001:00001f4c       exitOnError                0000000180002f4c f   libisobsolete001.obj
 0001:00002000       fprintf                    0000000180003000 f i libisobsolete001.obj
 0001:00002540       nsk_complain               0000000180003540 f   libisobsolete001.obj
 0001:0000256c       nsk_jvmti_createJVMTIEnv   000000018000356c f   libisobsolete001.obj
 0001:0000269c       nsk_jvmti_lverify          000000018000369c f   libisobsolete001.obj
 0001:0000278c       nsk_jvmti_parseOptions     000000018000378c f   libisobsolete001.obj
 0001:000029dc       nsk_jvmti_resetAgentData   00000001800039dc f   libisobsolete001.obj
 0001:00002a5c       nsk_jvmti_resumeSync       0000000180003a5c f   libisobsolete001.obj
 0001:00002b04       nsk_jvmti_setFailStatus    0000000180003b04 f   libisobsolete001.obj
 0001:00002b40       nsk_jvmti_threadByName     0000000180003b40 f   libisobsolete001.obj
 0001:00002e60       nsk_jvmti_waitForSync      0000000180003e60 f   libisobsolete001.obj
 0001:00002f64       nsk_lcomplain              0000000180003f64 f   libisobsolete001.obj
 0001:00002f84       nsk_ldisplay               0000000180003f84 f   libisobsolete001.obj
 0001:00002fa4       nsk_ltrace                 0000000180003fa4 f   libisobsolete001.obj
 0001:00002fc4       nsk_lvcomplain             0000000180003fc4 f   libisobsolete001.obj
 0001:0000317c       nsk_lvdisplay              000000018000417c f   libisobsolete001.obj
 0001:000031c8       nsk_lverify                00000001800041c8 f   libisobsolete001.obj
 0001:00003224       nsk_lvtrace                0000000180004224 f   libisobsolete001.obj
 0001:00003284       nsk_printf                 0000000180004284 f   libisobsolete001.obj
 0001:000032ac       nsk_vprintf                00000001800042ac f   libisobsolete001.obj
 0001:00003360       printf                     0000000180004360 f i libisobsolete001.obj
 0001:00003984       __raise_securityfailure    0000000180004984 f   MSVCRT:gs_report.obj
 0001:000039b8       __report_gsfailure         00000001800049b8 f   MSVCRT:gs_report.obj
 0001:00003bf8       __GSHandlerCheck           0000000180004bf8 f   MSVCRT:gshandler.obj
 0001:00003c18       __GSHandlerCheckCommon     0000000180004c18 f   MSVCRT:gshandler.obj
 0001:00003c90       __security_check_cookie    0000000180004c90 f   MSVCRT:amdsecgs.obj
 0001:00003fd0       _DllMainCRTStartup         0000000180004fd0 f   MSVCRT:dll_dllmain.obj
 0001:00004010       __scrt_acquire_startup_lock 0000000180005010 f   MSVCRT:utility.obj
 0001:0000404c       __scrt_dllmain_after_initialize_c 000000018000504c f   MSVCRT:utility.obj
 0001:00004080       __scrt_dllmain_before_initialize_c 0000000180005080 f   MSVCRT:utility.obj
 0001:00004098       __scrt_dllmain_crt_thread_attach 0000000180005098 f   MSVCRT:utility.obj
 0001:000040c0       __scrt_dllmain_crt_thread_detach 00000001800050c0 f   MSVCRT:utility.obj
 0001:000040d8       __scrt_dllmain_exception_filter 00000001800050d8 f   MSVCRT:utility.obj
 0001:00004138       __scrt_dllmain_uninitialize_c 0000000180005138 f   MSVCRT:utility.obj
 0001:00004168       __scrt_dllmain_uninitialize_critical 0000000180005168 f   MSVCRT:utility.obj
 0001:0000417c       __scrt_initialize_crt      000000018000517c f   MSVCRT:utility.obj
 0001:000041c8       __scrt_initialize_onexit_tables 00000001800051c8 f   MSVCRT:utility.obj
 0001:00004254       __scrt_is_nonwritable_in_current_image 0000000180005254 f   MSVCRT:utility.obj
 0001:000042ec       __scrt_release_startup_lock 00000001800052ec f   MSVCRT:utility.obj
 0001:00004310       __scrt_uninitialize_crt    0000000180005310 f   MSVCRT:utility.obj
 0001:0000433c       _onexit                    000000018000533c f   MSVCRT:utility.obj
 0001:00004378       atexit                     0000000180005378 f   MSVCRT:utility.obj
 0001:00004390       __crt_debugger_hook        0000000180005390 f   MSVCRT:utility_desktop.obj
 0001:00004398       __scrt_fastfail            0000000180005398 f   MSVCRT:utility_desktop.obj
 0001:000044e4       _guard_check_icall_nop     00000001800054e4 f i MSVCRT:guard_support.obj
 0001:000044e8       __security_init_cookie     00000001800054e8 f   MSVCRT:gs_support.obj
 0001:00004594       DllMain                    0000000180005594 f   MSVCRT:dll_dllmain_stub.obj
 0001:000045b8       ?__scrt_initialize_type_info@@YAXXZ 00000001800055b8 f   MSVCRT:tncleanup.obj
 0001:000045c8       ?__scrt_uninitialize_type_info@@YAXXZ 00000001800055c8 f   MSVCRT:tncleanup.obj
 0001:000045d4       __local_stdio_scanf_options 00000001800055d4 f i MSVCRT:default_local_stdio_options.obj
 0001:000045dc       __scrt_initialize_default_local_stdio_options 00000001800055dc f   MSVCRT:default_local_stdio_options.obj
 0001:000045f8       __scrt_get_dyn_tls_init_callback 00000001800055f8 f   MSVCRT:dyn_tls_init.obj
 0001:00004600       _RTC_Initialize            0000000180005600 f   MSVCRT:initsect.obj
 0001:0000463c       _RTC_Terminate             000000018000563c f   MSVCRT:initsect.obj
 0001:00004678       __isa_available_init       0000000180005678 f   MSVCRT:cpu_disp.obj
 0001:00004824       _get_startup_argv_mode     0000000180005824 f   MSVCRT:argv_mode.obj
 0001:0000482c       __scrt_is_ucrt_dll_in_use  000000018000582c f   MSVCRT:ucrt_detection.obj
 0001:00004840       memcpy                     0000000180005840 f   vcruntime:VCRUNTIME140.dll
 0001:00004846       memset                     0000000180005846 f   vcruntime:VCRUNTIME140.dll
 0001:0000484c       strchr                     000000018000584c f   vcruntime:VCRUNTIME140.dll
 0001:00004852       __C_specific_handler       0000000180005852 f   vcruntime:VCRUNTIME140.dll
 0001:00004858       __std_type_info_destroy_list 0000000180005858 f   vcruntime:VCRUNTIME140.dll
 0001:0000485e       strcmp                     000000018000585e f   ucrt:api-ms-win-crt-string-l1-1-0.dll
 0001:00004864       strlen                     0000000180005864 f   ucrt:api-ms-win-crt-string-l1-1-0.dll
 0001:0000486a       _initterm                  000000018000586a f   ucrt:api-ms-win-crt-runtime-l1-1-0.dll
 0001:00004870       _initterm_e                0000000180005870 f   ucrt:api-ms-win-crt-runtime-l1-1-0.dll
 0001:00004876       _seh_filter_dll            0000000180005876 f   ucrt:api-ms-win-crt-runtime-l1-1-0.dll
 0001:0000487c       _configure_narrow_argv     000000018000587c f   ucrt:api-ms-win-crt-runtime-l1-1-0.dll
 0001:00004882       _initialize_narrow_environment 0000000180005882 f   ucrt:api-ms-win-crt-runtime-l1-1-0.dll
 0001:00004888       _initialize_onexit_table   0000000180005888 f   ucrt:api-ms-win-crt-runtime-l1-1-0.dll
 0001:0000488e       _register_onexit_function  000000018000588e f   ucrt:api-ms-win-crt-runtime-l1-1-0.dll
 0001:00004894       _execute_onexit_table      0000000180005894 f   ucrt:api-ms-win-crt-runtime-l1-1-0.dll
 0001:0000489a       _crt_atexit                000000018000589a f   ucrt:api-ms-win-crt-runtime-l1-1-0.dll
 0001:000048a0       _cexit                     00000001800058a0 f   ucrt:api-ms-win-crt-runtime-l1-1-0.dll
 0001:000048a8       __acrt_initialize          00000001800058a8 f   MSVCRT:ucrt_stubs.obj
 0001:000048a8       __acrt_thread_attach       00000001800058a8 f   MSVCRT:ucrt_stubs.obj
 0001:000048a8       __acrt_thread_detach       00000001800058a8 f   MSVCRT:ucrt_stubs.obj
 0001:000048a8       __acrt_uninitialize        00000001800058a8 f   MSVCRT:ucrt_stubs.obj
 0001:000048a8       __acrt_uninitialize_critical 00000001800058a8 f   MSVCRT:ucrt_stubs.obj
 0001:000048a8       __scrt_stub_for_acrt_initialize 00000001800058a8 f   MSVCRT:ucrt_stubs.obj
 0001:000048a8       __scrt_stub_for_acrt_thread_attach 00000001800058a8 f   MSVCRT:ucrt_stubs.obj
 0001:000048a8       __scrt_stub_for_acrt_thread_detach 00000001800058a8 f   MSVCRT:ucrt_stubs.obj
 0001:000048a8       __scrt_stub_for_acrt_uninitialize 00000001800058a8 f   MSVCRT:ucrt_stubs.obj
 0001:000048a8       __scrt_stub_for_acrt_uninitialize_critical 00000001800058a8 f   MSVCRT:ucrt_stubs.obj
 0001:000048a8       __vcrt_initialize          00000001800058a8 f   MSVCRT:ucrt_stubs.obj
 0001:000048a8       __vcrt_thread_attach       00000001800058a8 f   MSVCRT:ucrt_stubs.obj
 0001:000048a8       __vcrt_thread_detach       00000001800058a8 f   MSVCRT:ucrt_stubs.obj
 0001:000048a8       __vcrt_uninitialize        00000001800058a8 f   MSVCRT:ucrt_stubs.obj
 0001:000048a8       __vcrt_uninitialize_critical 00000001800058a8 f   MSVCRT:ucrt_stubs.obj
 0001:000048ac       __scrt_stub_for_is_c_termination_complete 00000001800058ac f   MSVCRT:ucrt_stubs.obj
 0001:000048ac       _is_c_termination_complete 00000001800058ac f   MSVCRT:ucrt_stubs.obj
 0001:000048c0       _guard_dispatch_icall_nop  00000001800058c0 f   MSVCRT:guard_dispatch.obj
 0001:000048e0       _guard_xfg_dispatch_icall_nop 00000001800058e0 f   MSVCRT:guard_xfg_dispatch.obj
 0002:00000000       __imp_RtlCaptureContext    0000000180006000     kernel32:KERNEL32.dll
 0002:00000008       __imp_RtlLookupFunctionEntry 0000000180006008     kernel32:KERNEL32.dll
 0002:00000010       __imp_RtlVirtualUnwind     0000000180006010     kernel32:KERNEL32.dll
 0002:00000018       __imp_UnhandledExceptionFilter 0000000180006018     kernel32:KERNEL32.dll
 0002:00000020       __imp_SetUnhandledExceptionFilter 0000000180006020     kernel32:KERNEL32.dll
 0002:00000028       __imp_GetCurrentProcess    0000000180006028     kernel32:KERNEL32.dll
 0002:00000030       __imp_TerminateProcess     0000000180006030     kernel32:KERNEL32.dll
 0002:00000038       __imp_IsProcessorFeaturePresent 0000000180006038     kernel32:KERNEL32.dll
 0002:00000040       __imp_CloseHandle          0000000180006040     kernel32:KERNEL32.dll
 0002:00000048       __imp_InitializeCriticalSectionAndSpinCount 0000000180006048     kernel32:KERNEL32.dll
 0002:00000050       __imp_DeleteCriticalSection 0000000180006050     kernel32:KERNEL32.dll
 0002:00000058       __imp_CreateEventW         0000000180006058     kernel32:KERNEL32.dll
 0002:00000060       __imp_GetModuleHandleW     0000000180006060     kernel32:KERNEL32.dll
 0002:00000068       __imp_GetProcAddress       0000000180006068     kernel32:KERNEL32.dll
 0002:00000070       __imp_IsDebuggerPresent    0000000180006070     kernel32:KERNEL32.dll
 0002:00000078       __imp_QueryPerformanceCounter 0000000180006078     kernel32:KERNEL32.dll
 0002:00000080       __imp_GetCurrentProcessId  0000000180006080     kernel32:KERNEL32.dll
 0002:00000088       __imp_GetCurrentThreadId   0000000180006088     kernel32:KERNEL32.dll
 0002:00000090       __imp_GetSystemTimeAsFileTime 0000000180006090     kernel32:KERNEL32.dll
 0002:00000098       __imp_DisableThreadLibraryCalls 0000000180006098     kernel32:KERNEL32.dll
 0002:000000a0       __imp_InitializeSListHead  00000001800060a0     kernel32:KERNEL32.dll
 0002:000000a8       \177KERNEL32_NULL_THUNK_DATA 00000001800060a8     kernel32:KERNEL32.dll
 0002:000000b0       __imp_memcpy               00000001800060b0     vcruntime:VCRUNTIME140.dll
 0002:000000b8       __imp_memset               00000001800060b8     vcruntime:VCRUNTIME140.dll
 0002:000000c0       __imp_strchr               00000001800060c0     vcruntime:VCRUNTIME140.dll
 0002:000000c8       __imp___C_specific_handler 00000001800060c8     vcruntime:VCRUNTIME140.dll
 0002:000000d0       __imp___std_type_info_destroy_list 00000001800060d0     vcruntime:VCRUNTIME140.dll
 0002:000000d8       \177VCRUNTIME140_NULL_THUNK_DATA 00000001800060d8     vcruntime:VCRUNTIME140.dll
 0002:000000e0       __imp_strtol               00000001800060e0     ucrt:api-ms-win-crt-convert-l1-1-0.dll
 0002:000000e8       \177api-ms-win-crt-convert-l1-1-0_NULL_THUNK_DATA 00000001800060e8     ucrt:api-ms-win-crt-convert-l1-1-0.dll
 0002:000000f0       __imp_malloc               00000001800060f0     ucrt:api-ms-win-crt-heap-l1-1-0.dll
 0002:000000f8       __imp_free                 00000001800060f8     ucrt:api-ms-win-crt-heap-l1-1-0.dll
 0002:00000100       \177api-ms-win-crt-heap-l1-1-0_NULL_THUNK_DATA 0000000180006100     ucrt:api-ms-win-crt-heap-l1-1-0.dll
 0002:00000108       __imp__errno               0000000180006108     ucrt:api-ms-win-crt-runtime-l1-1-0.dll
 0002:00000110       __imp_exit                 0000000180006110     ucrt:api-ms-win-crt-runtime-l1-1-0.dll
 0002:00000118       __imp__cexit               0000000180006118     ucrt:api-ms-win-crt-runtime-l1-1-0.dll
 0002:00000120       __imp__crt_atexit          0000000180006120     ucrt:api-ms-win-crt-runtime-l1-1-0.dll
 0002:00000128       __imp__execute_onexit_table 0000000180006128     ucrt:api-ms-win-crt-runtime-l1-1-0.dll
 0002:00000130       __imp__register_onexit_function 0000000180006130     ucrt:api-ms-win-crt-runtime-l1-1-0.dll
 0002:00000138       __imp__initialize_onexit_table 0000000180006138     ucrt:api-ms-win-crt-runtime-l1-1-0.dll
 0002:00000140       __imp__initialize_narrow_environment 0000000180006140     ucrt:api-ms-win-crt-runtime-l1-1-0.dll
 0002:00000148       __imp__configure_narrow_argv 0000000180006148     ucrt:api-ms-win-crt-runtime-l1-1-0.dll
 0002:00000150       __imp__seh_filter_dll      0000000180006150     ucrt:api-ms-win-crt-runtime-l1-1-0.dll
 0002:00000158       __imp__initterm_e          0000000180006158     ucrt:api-ms-win-crt-runtime-l1-1-0.dll
 0002:00000160       __imp__initterm            0000000180006160     ucrt:api-ms-win-crt-runtime-l1-1-0.dll
 0002:00000168       \177api-ms-win-crt-runtime-l1-1-0_NULL_THUNK_DATA 0000000180006168     ucrt:api-ms-win-crt-runtime-l1-1-0.dll
 0002:00000170       __imp___acrt_iob_func      0000000180006170     ucrt:api-ms-win-crt-stdio-l1-1-0.dll
 0002:00000178       __imp_fflush               0000000180006178     ucrt:api-ms-win-crt-stdio-l1-1-0.dll
 0002:00000180       __imp___stdio_common_vsprintf 0000000180006180     ucrt:api-ms-win-crt-stdio-l1-1-0.dll
 0002:00000188       __imp___stdio_common_vfprintf 0000000180006188     ucrt:api-ms-win-crt-stdio-l1-1-0.dll
 0002:00000190       \177api-ms-win-crt-stdio-l1-1-0_NULL_THUNK_DATA 0000000180006190     ucrt:api-ms-win-crt-stdio-l1-1-0.dll
 0002:00000198       __imp_strcmp               0000000180006198     ucrt:api-ms-win-crt-string-l1-1-0.dll
 0002:000001a0       __imp__strdup              00000001800061a0     ucrt:api-ms-win-crt-string-l1-1-0.dll
 0002:000001a0       __imp_strdup               00000001800061a0     ucrt:api-ms-win-crt-string-l1-1-0.dll
 0002:000001a8       __imp_strlen               00000001800061a8     ucrt:api-ms-win-crt-string-l1-1-0.dll
 0002:000001b0       __imp_strpbrk              00000001800061b0     ucrt:api-ms-win-crt-string-l1-1-0.dll
 0002:000001b8       __imp_strncpy              00000001800061b8     ucrt:api-ms-win-crt-string-l1-1-0.dll
 0002:000001c0       \177api-ms-win-crt-string-l1-1-0_NULL_THUNK_DATA 00000001800061c0     ucrt:api-ms-win-crt-string-l1-1-0.dll
 0002:000001c8       __guard_check_icall_fptr   00000001800061c8     MSVCRT:guard_support.obj
 0002:000001d0       __guard_xfg_check_icall_fptr 00000001800061d0     MSVCRT:guard_support.obj
 0002:000001d8       __guard_dispatch_icall_fptr 00000001800061d8     MSVCRT:guard_support.obj
 0002:000001e0       __guard_xfg_dispatch_icall_fptr 00000001800061e0     MSVCRT:guard_support.obj
 0002:000001e8       __guard_xfg_table_dispatch_icall_fptr 00000001800061e8     MSVCRT:guard_support.obj
 0002:000001f0       __castguard_check_failure_os_handled_fptr 00000001800061f0     MSVCRT:guard_support.obj
 0002:000001f8       __guard_memcpy_fptr        00000001800061f8     vcruntime:softmemtag.obj
 0002:00000200       __xc_a                     0000000180006200     MSVCRT:initializers.obj
 0002:00000208       __xc_z                     0000000180006208     MSVCRT:initializers.obj
 0002:00000210       __xi_a                     0000000180006210     MSVCRT:initializers.obj
 0002:00000220       __xi_z                     0000000180006220     MSVCRT:initializers.obj
 0002:00000228       __xl_a                     0000000180006228     MSVCRT:tlssup.obj
 0002:00000230       __xl_z                     0000000180006230     MSVCRT:tlssup.obj
 0002:00000238       __xp_a                     0000000180006238     MSVCRT:initializers.obj
 0002:00000240       __xp_z                     0000000180006240     MSVCRT:initializers.obj
 0002:00000248       __xt_a                     0000000180006248     MSVCRT:initializers.obj
 0002:00000250       __xt_z                     0000000180006250     MSVCRT:initializers.obj
 0002:00000260       g_refKindStr               0000000180006260     libisobsolete001.obj
 0002:00000410       ??_C@_09BPLDFGCI@unknown_0@ 0000000180006410     libisobsolete001.obj
 0002:00000420       ??_C@_0BL@FPNMECJD@JVMTI_HEAP_REFERENCE_CLASS@ 0000000180006420     libisobsolete001.obj
 0002:00000440       ??_C@_0BL@FKGKKLNM@JVMTI_HEAP_REFERENCE_FIELD@ 0000000180006440     libisobsolete001.obj
 0002:00000460       ??_C@_0CD@CAEHCFJF@JVMTI_HEAP_REFERENCE_ARRAY_ELEM@ 0000000180006460     libisobsolete001.obj
 0002:00000488       ??_C@_0CC@DNEBMCNK@JVMTI_HEAP_REFERENCE_CLASS_LOAD@ 0000000180006488     libisobsolete001.obj
 0002:000004b0       ??_C@_0BN@CJMIPEBB@JVMTI_HEAP_REFERENCE_SIGNERS@ 00000001800064b0     libisobsolete001.obj
 0002:000004d0       ??_C@_0CH@HBOIDPEB@JVMTI_HEAP_REFERENCE_PROTECTION@ 00000001800064d0     libisobsolete001.obj
 0002:000004f8       ??_C@_0BP@MDKGDGKL@JVMTI_HEAP_REFERENCE_INTERFACE@ 00000001800064f8     libisobsolete001.obj
 0002:00000518       ??_C@_0CC@JJMIHNJH@JVMTI_HEAP_REFERENCE_STATIC_FIE@ 0000000180006518     libisobsolete001.obj
 0002:00000540       ??_C@_0CD@IDHEEGID@JVMTI_HEAP_REFERENCE_CONSTANT_P@ 0000000180006540     libisobsolete001.obj
 0002:00000568       ??_C@_0CA@EFFCHNG@JVMTI_HEAP_REFERENCE_SUPERCLASS@ 0000000180006568     libisobsolete001.obj
 0002:00000588       ??_C@_0L@PCDFHGCJ@unknown_11@ 0000000180006588     libisobsolete001.obj
 0002:00000598       ??_C@_0L@NJBICFOK@unknown_12@ 0000000180006598     libisobsolete001.obj
 0002:000005a8       ??_C@_0L@MAADBEKL@unknown_13@ 00000001800065a8     libisobsolete001.obj
 0002:000005b8       ??_C@_0L@IPECICGM@unknown_14@ 00000001800065b8     libisobsolete001.obj
 0002:000005c8       ??_C@_0L@JGFJLDCN@unknown_15@ 00000001800065c8     libisobsolete001.obj
 0002:000005d8       ??_C@_0L@LNHEOAOO@unknown_16@ 00000001800065d8     libisobsolete001.obj
 0002:000005e8       ??_C@_0L@KEGPNBKP@unknown_17@ 00000001800065e8     libisobsolete001.obj
 0002:000005f8       ??_C@_0L@CDPHMNGA@unknown_18@ 00000001800065f8     libisobsolete001.obj
 0002:00000608       ??_C@_0L@DKOMPMCB@unknown_19@ 0000000180006608     libisobsolete001.obj
 0002:00000618       ??_C@_0L@OJGIPJDB@unknown_20@ 0000000180006618     libisobsolete001.obj
 0002:00000628       ??_C@_0CA@KAOFNDEM@JVMTI_HEAP_REFERENCE_JNI_GLOBAL@ 0000000180006628     libisobsolete001.obj
 0002:00000648       ??_C@_0CC@HPFAJBK@JVMTI_HEAP_REFERENCE_SYSTEM_CLA@ 0000000180006648     libisobsolete001.obj
 0002:00000670       ??_C@_0BN@FDEGFOHC@JVMTI_HEAP_REFERENCE_MONITOR@ 0000000180006670     libisobsolete001.obj
 0002:00000690       ??_C@_0CB@HKIBCMAJ@JVMTI_HEAP_REFERENCE_STACK_LOCA@ 0000000180006690     libisobsolete001.obj
 0002:000006b8       ??_C@_0BP@EAACMMOE@JVMTI_HEAP_REFERENCE_JNI_LOCAL@ 00000001800066b8     libisobsolete001.obj
 0002:000006d8       ??_C@_0BM@IJDEOGOE@JVMTI_HEAP_REFERENCE_THREAD@ 00000001800066d8     libisobsolete001.obj
 0002:000006f8       ??_C@_0BL@EDGPPKC@JVMTI_HEAP_REFERENCE_OTHER@ 00000001800066f8     libisobsolete001.obj
 0002:00000714       ??_C@_04BCJPDBDA@Code@     0000000180006714     libisobsolete001.obj
 0002:00000720       ??_C@_0BA@OCLMCFKC@LineNumberTable@ 0000000180006720     libisobsolete001.obj
 0002:00000730       ??_C@_0BD@CPAEPILC@LocalVariableTable@ 0000000180006730     libisobsolete001.obj
 0002:00000748       ??_C@_0BH@NMBDNHBD@LocalVariableTypeTable@ 0000000180006748     libisobsolete001.obj
 0002:00000760       ??_C@_0O@HIHEEDNJ@StackMapTable@ 0000000180006760     libisobsolete001.obj
 0002:00000770       ??_C@_0L@HCDIAMJG@?9?5?$CFs?0?5?$CFd?3?5@ 0000000180006770     libisobsolete001.obj
 0002:00000780       ??_C@_0JI@HLPECLFI@?$CD?5?4?4?4?6?$CD?5ERROR?3?5too?5many?5complai@ 0000000180006780     libisobsolete001.obj
 0002:00000820       ??_C@_0ED@JNEKCCOB@The?5following?5fake?5exception?5st@ 0000000180006820     libisobsolete001.obj
 0002:00000868       ??_C@_0CN@FCNMDFBH@nsk?4share?4Fake_Exception_for_RU@ 0000000180006868     libisobsolete001.obj
 0002:00000898       ??_C@_08PGFFNAEI@?$CI?$CFs?3?$CFd?$CJ?5@ 0000000180006898     libisobsolete001.obj
 0002:000008a8       ??_C@_0DP@IENMAEGI@s?2test?2hotspot?2jtreg?2vmTestbase@ 00000001800068a8     libisobsolete001.obj
 0002:000008e8       ??_C@_0BL@NDJLFFJB@?7at?5nsk_lvcomplain?$CI?$CFs?3?$CFd?$CJ?6@ 00000001800068e8     libisobsolete001.obj
 0002:00000908       ??_C@_0BC@JOOKAFKF@?$CD?5ERROR?3?5?$CFs?0?5?$CFd?3?5@ 0000000180006908     libisobsolete001.obj
 0002:00000920       ??_C@_09KJEAHMEH@?$CD?5ERROR?3?5@ 0000000180006920     libisobsolete001.obj
 0002:0000092c       ??_C@_02GPIOPFAK@?$DO?$DO@ 000000018000692c     libisobsolete001.obj
 0002:00000930       ??_C@_02FODMEDOG@?$DM?$DM@ 0000000180006930     libisobsolete001.obj
 0002:00000934       ??_C@_02DJGKEECL@?4?4@     0000000180006934     libisobsolete001.obj
 0002:00000938       ??_C@_0O@CJPGJOAF@?9?5?$CFs?0?5?$CFd?3?5?$CFs?5@ 0000000180006938     libisobsolete001.obj
 0002:00000948       ??_C@_0CB@IAKPDOIC@?$CD?5?5?5verified?5assertion?5is?5FALSE@ 0000000180006948     libisobsolete001.obj
 0002:00000970       ??_C@_0CO@LGONDEPD@stdout?3?5fflush?5failed?5?9?5err?$DN?$CFd?5@ 0000000180006970     libisobsolete001.obj
 0002:000009a0       ??_C@_0CO@KBGKJPBD@stderr?3?5fflush?5failed?5?9?5err?$DN?$CFd?5@ 00000001800069a0     libisobsolete001.obj
 0002:000009d0       ??_C@_06HPGEIPLA@?$DMnull?$DO@ 00000001800069d0     libisobsolete001.obj
 0002:000009d8       ??_C@_0BB@JCNMKLLK@JVMTI_ERROR_NONE@ 00000001800069d8     libisobsolete001.obj
 0002:000009f0       ??_C@_0BL@LDIMKLPH@JVMTI_ERROR_INVALID_THREAD@ 00000001800069f0     libisobsolete001.obj
 0002:00000a10       ??_C@_0CB@PJFPAIKJ@JVMTI_ERROR_INVALID_THREAD_GROU@ 0000000180006a10     libisobsolete001.obj
 0002:00000a38       ??_C@_0BN@LLMKHMNF@JVMTI_ERROR_INVALID_PRIORITY@ 0000000180006a38     libisobsolete001.obj
 0002:00000a58       ??_C@_0CB@MBOFKAGB@JVMTI_ERROR_THREAD_NOT_SUSPENDE@ 0000000180006a58     libisobsolete001.obj
 0002:00000a80       ??_C@_0BN@FABOLPBI@JVMTI_ERROR_THREAD_SUSPENDED@ 0000000180006a80     libisobsolete001.obj
 0002:00000aa0       ??_C@_0BN@FDGNOBJM@JVMTI_ERROR_THREAD_NOT_ALIVE@ 0000000180006aa0     libisobsolete001.obj
 0002:00000ac0       ??_C@_0BL@GOBIFKNJ@JVMTI_ERROR_INVALID_OBJECT@ 0000000180006ac0     libisobsolete001.obj
 0002:00000ae0       ??_C@_0BK@FCMAJPPC@JVMTI_ERROR_INVALID_CLASS@ 0000000180006ae0     libisobsolete001.obj
 0002:00000b00       ??_C@_0BP@IKLLBKEB@JVMTI_ERROR_CLASS_NOT_PREPARED@ 0000000180006b00     libisobsolete001.obj
 0002:00000b20       ??_C@_0BN@KLPPLKG@JVMTI_ERROR_INVALID_METHODID@ 0000000180006b20     libisobsolete001.obj
 0002:00000b40       ??_C@_0BN@BCEKOKND@JVMTI_ERROR_INVALID_LOCATION@ 0000000180006b40     libisobsolete001.obj
 0002:00000b60       ??_C@_0BM@DFDGPME@JVMTI_ERROR_INVALID_FIELDID@ 0000000180006b60     libisobsolete001.obj
 0002:00000b80       ??_C@_0BL@NELIEPEC@JVMTI_ERROR_NO_MORE_FRAMES@ 0000000180006b80     libisobsolete001.obj
 0002:00000ba0       ??_C@_0BJ@BDBECFDM@JVMTI_ERROR_OPAQUE_FRAME@ 0000000180006ba0     libisobsolete001.obj
 0002:00000bc0       ??_C@_0BK@MIIFNLOB@JVMTI_ERROR_TYPE_MISMATCH@ 0000000180006bc0     libisobsolete001.obj
 0002:00000be0       ??_C@_0BJ@HPCAOILC@JVMTI_ERROR_INVALID_SLOT@ 0000000180006be0     libisobsolete001.obj
 0002:00000c00       ??_C@_0BG@CHILOPNI@JVMTI_ERROR_DUPLICATE@ 0000000180006c00     libisobsolete001.obj
 0002:00000c18       ??_C@_0BG@DIEMLHKM@JVMTI_ERROR_NOT_FOUND@ 0000000180006c18     libisobsolete001.obj
 0002:00000c30       ??_C@_0BM@NHMCKHOB@JVMTI_ERROR_INVALID_MONITOR@ 0000000180006c30     libisobsolete001.obj
 0002:00000c50       ??_C@_0BO@PPEDAJGL@JVMTI_ERROR_NOT_MONITOR_OWNER@ 0000000180006c50     libisobsolete001.obj
 0002:00000c70       ??_C@_0BG@FCAIPEID@JVMTI_ERROR_INTERRUPT@ 0000000180006c70     libisobsolete001.obj
 0002:00000c88       ??_C@_0CB@EGDBNKOI@JVMTI_ERROR_INVALID_CLASS_FORMA@ 0000000180006c88     libisobsolete001.obj
 0002:00000cb0       ??_C@_0CG@DGKOGIAL@JVMTI_ERROR_CIRCULAR_CLASS_DEFI@ 0000000180006cb0     libisobsolete001.obj
 0002:00000cd8       ??_C@_0BP@ICEALPKC@JVMTI_ERROR_FAILS_VERIFICATION@ 0000000180006cd8     libisobsolete001.obj
 0002:00000cf8       ??_C@_0DC@JDACLMIO@JVMTI_ERROR_UNSUPPORTED_REDEFIN@ 0000000180006cf8     libisobsolete001.obj
 0002:00000d30       ??_C@_0DE@GKDKNOMJ@JVMTI_ERROR_UNSUPPORTED_REDEFIN@ 0000000180006d30     libisobsolete001.obj
 0002:00000d68       ??_C@_0BO@LAFKIOG@JVMTI_ERROR_INVALID_TYPESTATE@ 0000000180006d68     libisobsolete001.obj
 0002:00000d88       ??_C@_0DH@INDGCLLB@JVMTI_ERROR_UNSUPPORTED_REDEFIN@ 0000000180006d88     libisobsolete001.obj
 0002:00000dc0       ??_C@_0DE@NHEOMMGI@JVMTI_ERROR_UNSUPPORTED_REDEFIN@ 0000000180006dc0     libisobsolete001.obj
 0002:00000df8       ??_C@_0CA@EKPNJOEP@JVMTI_ERROR_UNSUPPORTED_VERSION@ 0000000180006df8     libisobsolete001.obj
 0002:00000e18       ??_C@_0BN@OFFMAHHL@JVMTI_ERROR_NAMES_DONT_MATCH@ 0000000180006e18     libisobsolete001.obj
 0002:00000e38       ??_C@_0DN@HHBBLAKE@JVMTI_ERROR_UNSUPPORTED_REDEFIN@ 0000000180006e38     libisobsolete001.obj
 0002:00000e78       ??_C@_0DO@HMBGBGNA@JVMTI_ERROR_UNSUPPORTED_REDEFIN@ 0000000180006e78     libisobsolete001.obj
 0002:00000eb8       ??_C@_0BP@PBECGKHJ@JVMTI_ERROR_UNMODIFIABLE_CLASS@ 0000000180006eb8     libisobsolete001.obj
 0002:00000ed8       ??_C@_0BK@CANILEHF@JVMTI_ERROR_NOT_AVAILABLE@ 0000000180006ed8     libisobsolete001.obj
 0002:00000ef8       ??_C@_0CE@INJKMEFK@JVMTI_ERROR_MUST_POSSESS_CAPABI@ 0000000180006ef8     libisobsolete001.obj
 0002:00000f20       ??_C@_0BJ@LBFPFPDM@JVMTI_ERROR_NULL_POINTER@ 0000000180006f20     libisobsolete001.obj
 0002:00000f40       ??_C@_0BP@CHJPNNEM@JVMTI_ERROR_ABSENT_INFORMATION@ 0000000180006f40     libisobsolete001.obj
 0002:00000f60       ??_C@_0BP@OMFMNLC@JVMTI_ERROR_INVALID_EVENT_TYPE@ 0000000180006f60     libisobsolete001.obj
 0002:00000f80       ??_C@_0BN@BIBNPHHO@JVMTI_ERROR_ILLEGAL_ARGUMENT@ 0000000180006f80     libisobsolete001.obj
 0002:00000fa0       ??_C@_0BK@KKNDHDCE@JVMTI_ERROR_NATIVE_METHOD@ 0000000180006fa0     libisobsolete001.obj
 0002:00000fc0       ??_C@_0BK@PMKCFHAE@JVMTI_ERROR_OUT_OF_MEMORY@ 0000000180006fc0     libisobsolete001.obj
 0002:00000fe0       ??_C@_0BK@NNJBDMNB@JVMTI_ERROR_ACCESS_DENIED@ 0000000180006fe0     libisobsolete001.obj
 0002:00001000       ??_C@_0BI@GHECLMNC@JVMTI_ERROR_WRONG_PHASE@ 0000000180007000     libisobsolete001.obj
 0002:00001018       ??_C@_0BF@OLIHJOII@JVMTI_ERROR_INTERNAL@ 0000000180007018     libisobsolete001.obj
 0002:00001030       ??_C@_0BO@EOHGKJHI@JVMTI_ERROR_UNATTACHED_THREAD@ 0000000180007030     libisobsolete001.obj
 0002:00001050       ??_C@_0CA@LKHFDACL@JVMTI_ERROR_INVALID_ENVIRONMENT@ 0000000180007050     libisobsolete001.obj
 0002:00001070       ??_C@_0BA@MMFHLOKK@?$DMunknown?5error?$DO@ 0000000180007070     libisobsolete001.obj
 0002:00001080       ??_C@_0CF@CBHOKDB@throwable?5?$DN?5jni?9?$DOExceptionOccur@ 0000000180007080     libisobsolete001.obj
 0002:000010a8       ??_C@_03OFAPEBGM@?$CFs?6@  00000001800070a8     libisobsolete001.obj
 0002:000010b0       ??_C@_0DM@LPIGEGNJ@s?2test?2hotspot?2jtreg?2vmTestbase@ 00000001800070b0     libisobsolete001.obj
 0002:000010f0       ??_C@_0CC@NFCNPEPK@Exception?5in?5JNI?5call?5?$CIcleared?$CJ@ 00000001800070f0     libisobsolete001.obj
 0002:00001118       ??_C@_0BJ@IBAKFIKF@jni?9?$DOExceptionDescribe?$CI?$CJ@ 0000000180007118     libisobsolete001.obj
 0002:00001138       ??_C@_0BG@GGKALKMH@jni?9?$DOExceptionClear?$CI?$CJ@ 0000000180007138     libisobsolete001.obj
 0002:00001150       ??_C@_0CF@JMGFGJLJ@?$CD?5?5?5verified?5JNI?5assertion?5is?5F@ 0000000180007150     libisobsolete001.obj
 0002:00001178       ??_C@_07KBAMPNJK@verbose@  0000000180007178     libisobsolete001.obj
 0002:00001180       ??_C@_0DN@PKJBOLAP@nsk_jvmti_parseOptions?$CI?$CJ?3?5unexp@ 0000000180007180     libisobsolete001.obj
 0002:000011c0       ??_C@_05IMBNNINJ@trace@    00000001800071c0     libisobsolete001.obj
 0002:000011c8       ??_C@_0DD@BJKGNDMB@nsk_jvmti_parseOptions?$CI?$CJ?3?5no?5va@ 00000001800071c8     libisobsolete001.obj
 0002:000011fc       ??_C@_04CGFJFPFD@none@     00000001800071fc     libisobsolete001.obj
 0002:00001204       ??_C@_06BMELKFMA@before@   0000000180007204     libisobsolete001.obj
 0002:0000120c       ??_C@_05CMKPCFDK@after@    000000018000720c     libisobsolete001.obj
 0002:00001214       ??_C@_03NFKEKGGK@all@      0000000180007214     libisobsolete001.obj
 0002:00001218       ??_C@_0DM@NDNJGJKE@nsk_jvmti_parseOptions?$CI?$CJ?3?5uexpe@ 0000000180007218     libisobsolete001.obj
 0002:00001258       ??_C@_08NBBJKJO@waittime@  0000000180007258     libisobsolete001.obj
 0002:00001268       ??_C@_0DO@CMHGAOHC@nsk_jvmti_parseOptions?$CI?$CJ?3?5not?5i@ 0000000180007268     libisobsolete001.obj
 0002:000012a8       ??_C@_0DL@LNMPBDLN@nsk_jvmti_parseOptions?$CI?$CJ?3?5negat@ 00000001800072a8     libisobsolete001.obj
 0002:000012e8       ??_C@_0DA@GMFJNOJH@nsk_jvmti_parseOptions?$CI?$CJ?3?5unkno@ 00000001800072e8     libisobsolete001.obj
 0002:00001318       ??_C@_0CO@CCIAMEAN@nsk_jvmti_parseOptions?$CI?$CJ?3?5found@ 0000000180007318     libisobsolete001.obj
 0002:00001348       ??_C@_0CJ@OEGPCGDL@nsk_jvmti_parseOptions?$CI?$CJ?3?5out?5o@ 0000000180007348     libisobsolete001.obj
 0002:00001378       ??_C@_0DI@NMBHPGGF@nsk_jvmti_parseOptions?$CI?$CJ?3?5too?5m@ 0000000180007378     libisobsolete001.obj
 0002:000013b0       ??_C@_03POGCGECB@?5?0?$HO@ 00000001800073b0     libisobsolete001.obj
 0002:000013b8       ??_C@_0CB@MLNJNCLJ@?5?5jvmti?5error?3?5code?$DN?$CFd?0?5name?$DN?$CFs@ 00000001800073b8     libisobsolete001.obj
 0002:000013e0       ??_C@_0CD@OHBGDKMK@?$CD?5?5?5jvmti?5error?3?5code?$DN?$CFd?0?5name?$DN@ 00000001800073e0     libisobsolete001.obj
 0002:00001408       ??_C@_0CG@JNNCGPHB@?$CD?5?5?5error?5expected?3?5code?$DN?$CFd?0?5na@ 0000000180007408     libisobsolete001.obj
 0002:00001430       ??_C@_0EB@IMGKPCGE@?$CIstr_obj?5?$DN?5jni?9?$DONewStringUTF?$CIco@ 0000000180007430     libisobsolete001.obj
 0002:00001480       ??_C@_0EA@HFOGGBCC@s?2test?2hotspot?2jtreg?2vmTestbase@ 0000000180007480     libisobsolete001.obj
 0002:000014c0       ??_C@_05KKCIMGE@error@     00000001800074c0     libisobsolete001.obj
 0002:000014c8       ??_C@_0CJ@JACLEAA@Test?5failed?5by?5setFailStatus?$CI?$CJ?4@ 00000001800074c8     libisobsolete001.obj
 0002:000014f8       ??_C@_0BD@HGNAOMCP@agent_data_monitor@ 00000001800074f8     libisobsolete001.obj
 0002:00001510       ??_C@_0EB@OGCLGKLN@javaVM?9?$DOGetEnv?$CI?$CIvoid?5?$CK?$CK?$CJ?$CGjvmti_@ 0000000180007510     libisobsolete001.obj
 0002:00001560       ??_C@_0EA@PNBCDMOA@s?2test?2hotspot?2jtreg?2vmTestbase@ 0000000180007560     libisobsolete001.obj
 0002:000015a0       ??_C@_0CI@DDPIFBGM@init_agent_data?$CIjvmti_env?0?5?$CGage@ 00000001800075a0     libisobsolete001.obj
 0002:000015c8       ??_C@_0DI@ILAHDLMP@?$CI?$CKagentThreadProc?$CJ?$CIjvmti_env?0?5a@ 00000001800075c8     libisobsolete001.obj
 0002:00001600       ??_C@_0BD@KDBALNLB@JVMTI?5agent?5thread@ 0000000180007600     libisobsolete001.obj
 0002:00001618       ??_C@_0BB@NOKBFPFO@java?1lang?1Thread@ 0000000180007618     libisobsolete001.obj
 0002:0000162c       ??_C@_06FALKBLGB@?$DMinit?$DO@ 000000018000762c     libisobsolete001.obj
 0002:00001638       ??_C@_0BG@IKDDPPGD@?$CILjava?1lang?1String?$DL?$CJV@ 0000000180007638     libisobsolete001.obj
 0002:00001650       ??_C@_0EB@IFJBFEKC@?$CIthreadClass?5?$DN?5jni_env?9?$DOFindCla@ 0000000180007650     libisobsolete001.obj
 0002:000016a0       ??_C@_0GF@FGFIBKKL@?$CIthreadCtor?5?$DN?5jni_env?9?$DOGetMetho@ 00000001800076a0     libisobsolete001.obj
 0002:00001708       ??_C@_0DN@NCPDJLOG@?$CIthreadName?5?$DN?5jni_env?9?$DONewStrin@ 0000000180007708     libisobsolete001.obj
 0002:00001750       ??_C@_0FE@PFKODBGC@?$CIthreadObject?5?$DN?5jni_env?9?$DONewObj@ 0000000180007750     libisobsolete001.obj
 0002:000017b0       ??_C@_0ED@HOBAHHJI@?$CIthreadGlobalRef?5?$DN?5jni_env?9?$DONew@ 00000001800077b0     libisobsolete001.obj
 0002:00001800       ??_C@_0FN@HNJJAHFC@jvmti_env?9?$DORunAgentThread?$CIagent@ 0000000180007800     libisobsolete001.obj
 0002:00001860       ??_C@_0EA@MOJDNKDF@Debuggee?5status?5sync?5aborted?5be@ 0000000180007860     libisobsolete001.obj
 0002:000018a0       ??_C@_0CO@PGPGMHBJ@No?5status?5sync?5occured?5for?5time@ 00000001800078a0     libisobsolete001.obj
 0002:000018d0       ??_C@_0CL@DOEBDPKJ@Debuggee?5was?5not?5suspended?5on?5s@ 00000001800078d0     libisobsolete001.obj
 0002:00001900       ??_C@_0EA@EEOEJAEN@status?5?$DN?5syncDebuggeeStatus?$CIjni@ 0000000180007900     libisobsolete001.obj
 0002:00001940       ??_C@_0BL@JBCFNBMB@nsk_jvmti_resetAgentData?$CI?$CJ@ 0000000180007940     libisobsolete001.obj
 0002:00001960       ??_C@_0BA@OEGNKEHK@name?5?$CB?$DN?5nullptr@ 0000000180007960     libisobsolete001.obj
 0002:00001970       ??_C@_0CL@BAHDCEOM@jvmti_env?9?$DOGetAllThreads?$CI?$CGcount@ 0000000180007970     libisobsolete001.obj
 0002:000019a0       ??_C@_0CM@KHOAGNIJ@jvmti_env?9?$DOGetThreadInfo?$CIthread@ 00000001800079a0     libisobsolete001.obj
 0002:000019d0       ??_C@_0DB@JOGMPONN@jvmti_env?9?$DODeallocate?$CI?$CIunsigned@ 00000001800079d0     libisobsolete001.obj
 0002:00001a08       ??_C@_0CP@KMNIFKEK@jvmti_env?9?$DODeallocate?$CI?$CIunsigned@ 0000000180007a08     libisobsolete001.obj
 0002:00001a40       ??_C@_0EI@EJCFGEKG@?$CIfoundThread?5?$DN?5?$CIjthread?$CJ?5jni_en@ 0000000180007a40     libisobsolete001.obj
 0002:00001a88       ??_C@_04DIFHPCLD@?$CII?$CJI@ 0000000180007a88     libisobsolete001.obj
 0002:00001a90       ??_C@_0EL@LPBEELIP@s?2test?2hotspot?2jtreg?2vmTestbase@ 0000000180007a90     libisobsolete001.obj
 0002:00001ae0       ??_C@_0CK@JDAMFDMJ@jvmti?9?$DOSetTag?$CIo?0?5tag?$CJ?5?$DN?$DN?5JVMTI_@ 0000000180007ae0     libisobsolete001.obj
 0002:00001b10       ??_C@_0CC@DAMNHKNI@Can?8t?5set?5tag?5?$CFli?5for?5object?5?$CFl@ 0000000180007b10     libisobsolete001.obj
 0002:00001b38       ??_C@_0DL@HAJPNKEF@jvmti?9?$DOGetObjectHashCode?$CIo?0?5?$CGha@ 0000000180007b38     libisobsolete001.obj
 0002:00001b78       ??_C@_0BL@JFPIEOBF@Can?8t?5get?5hash?5object?5?$CFlx?6@ 0000000180007b78     libisobsolete001.obj
 0002:00001b98       ??_C@_0BG@DICPHBKN@setTag?3?5?$CF08x?5?$DM?9?5?$CF?53li@ 0000000180007b98     libisobsolete001.obj
 0002:00001bb0       ??_C@_0DH@FCEEBDMJ@?$CIs?5?$DN?5jni?9?$DOGetStringUTFChars?$CIsIn@ 0000000180007bb0     libisobsolete001.obj
 0002:00001be8       ??_C@_0BJ@OKKGHDCN@Can?8t?5get?5string?5at?5?$CF?$CDp?6@ 0000000180007be8     libisobsolete001.obj
 0002:00001c08       ??_C@_0BP@EKFLGGFJ@Can?8t?5get?5string?5at?5?$CF?$CDp?3?5null?6@ 0000000180007c08     libisobsolete001.obj
 0002:00001c28       ??_C@_06ICODBHCL@?5?1?1?5?$CFs@ 0000000180007c28     libisobsolete001.obj
 0002:00001c30       ??_C@_0DB@KGFPLEGO@?$CIr?5?$DN?5jvmti?9?$DOGetTag?$CIo?0?5?$CGtag?$CJ?$CJ?5?$DN?$DN@ 0000000180007c30     libisobsolete001.obj
 0002:00001c68       ??_C@_0CO@PDAGBCGJ@Can?8t?5GetTag?5for?5object?5?$CFlx?4?5Re@ 0000000180007c68     libisobsolete001.obj
 0002:00001c98       ??_C@_0CH@HPEODOHC@TEST_BUG?3?5Max?4?5number?5of?5refs?5r@ 0000000180007c98     libisobsolete001.obj
 0002:00001cc0       ??_C@_0DI@PHFCABIM@?$CIr?5?$DN?5jvmti?9?$DOGetTag?$CIfrom?0?5?$CGtagFr@ 0000000180007cc0     libisobsolete001.obj
 0002:00001cf8       ??_C@_0DI@MDEGFNKD@TEST_BUG?3?5Can?8t?5GetTag?5for?5obje@ 0000000180007cf8     libisobsolete001.obj
 0002:00001d30       ??_C@_0DE@MLELJAHM@?$CIr?5?$DN?5jvmti?9?$DOGetTag?$CIto?0?5?$CGtagTo?$CJ?$CJ@ 0000000180007d30     libisobsolete001.obj
 0002:00001d68       ??_C@_0CK@JBPNHKIL@Call?5IsObsolete?$CI?$CJ?5for?5?$CFs?5method@ 0000000180007d68     libisobsolete001.obj
 0002:00001da0       ??_C@_0FL@NKDPPHPN@s?2test?2hotspot?2jtreg?2vmTestbase@ 0000000180007da0     libisobsolete001.obj
 0002:00001e00       ??_C@_0CL@IJJDPFMM@jvmti?9?$DOIsMethodObsolete?$CImethod?0@ 0000000180007e00     libisobsolete001.obj
 0002:00001e30       ??_C@_0BI@PMOPGMDJ@?5?5?4?4?4?5got?5obsolete?3?5?$CFd?6@ 0000000180007e30     libisobsolete001.obj
 0002:00001e50       ??_C@_0GD@GDLIOHBK@IsObsolete?$CI?$CJ?5returns?5unexpected@ 0000000180007e50     libisobsolete001.obj
 0002:00001eb8       ??_C@_0CB@GNANDEO@Get?5stack?5frames?5for?5thread?3?5?$CFp@ 0000000180007eb8     libisobsolete001.obj
 0002:00001ee0       ??_C@_0EK@NIFAIMNP@jvmti?9?$DOGetStackTrace?$CIthread?0?50?0@ 0000000180007ee0     libisobsolete001.obj
 0002:00001f30       ??_C@_0BG@PAFJAODF@?5?5?4?4?4?5got?5frames?3?5?$CFd?6@ 0000000180007f30     libisobsolete001.obj
 0002:00001f48       ??_C@_0CI@DLBGBKEO@Check?5methods?5of?5each?5frame?3?5?$CFd@ 0000000180007f48     libisobsolete001.obj
 0002:00001f70       ??_C@_0O@OIOEOOJI@?5?5frame?5?$CD?$CFi?3?6@ 0000000180007f70     libisobsolete001.obj
 0002:00001f80       ??_C@_0BE@HNJPNJNC@?5?5?5?5?5methodID?3?5?5?$CFp?6@ 0000000180007f80     libisobsolete001.obj
 0002:00001fa0       ??_C@_0EI@BOLEIPGC@jvmti?9?$DOGetMethodName?$CIframeStack@ 0000000180007fa0     libisobsolete001.obj
 0002:00001fe8       ??_C@_0BE@CDECKDLH@?5?5?5?5?5name?3?5?5?5?5?5?5?$CFs?6@ 0000000180007fe8     libisobsolete001.obj
 0002:00002000       ??_C@_0BE@JDGCGFBJ@?5?5?5?5?5signature?3?5?$CFs?6@ 0000000180008000     libisobsolete001.obj
 0002:00002018       ??_C@_0BE@PFBGJBOM@?5?5?5?5?5generic?3?5?5?5?$CFs?6@ 0000000180008018     libisobsolete001.obj
 0002:00002030       ??_C@_0BD@PBLOIOEE@testedStaticMethod@ 0000000180008030     libisobsolete001.obj
 0002:00002048       ??_C@_0BF@EGDBDJKJ@testedInstanceMethod@ 0000000180008048     libisobsolete001.obj
 0002:00002060       ??_C@_0CO@FNPFHBNC@SUCCESS?3?5found?5redefined?5method@ 0000000180008060     libisobsolete001.obj
 0002:00002090       ??_C@_0BD@JLHHOLAL@obsolete?5redefined@ 0000000180008090     libisobsolete001.obj
 0002:000020a8       ??_C@_0CI@BEMPBPFM@jvmti?9?$DODeallocate?$CI?$CIunsigned?5cha@ 00000001800080a8     libisobsolete001.obj
 0002:000020d0       ??_C@_0CN@OCDMNJJK@jvmti?9?$DODeallocate?$CI?$CIunsigned?5cha@ 00000001800080d0     libisobsolete001.obj
 0002:00002100       ??_C@_0CL@LNBMAIIC@jvmti?9?$DODeallocate?$CI?$CIunsigned?5cha@ 0000000180008100     libisobsolete001.obj
 0002:00002130       ??_C@_0FA@FAADFFBD@Not?5all?5?$CFs?5methods?5found?5on?5sta@ 0000000180008130     libisobsolete001.obj
 0002:00002180       ??_C@_0BE@CKPNMDMJ@Redefine?5class?3?5?$CFs?6@ 0000000180008180     libisobsolete001.obj
 0002:00002198       ??_C@_0CF@OBOBAJEI@jvmti?9?$DORedefineClasses?$CI1?0?5?$CGclas@ 0000000180008198     libisobsolete001.obj
 0002:000021c0       ??_C@_0CL@ODFFGLLA@?5?5?5?4?4?4?5redefined?5with?5classfile@ 00000001800081c0     libisobsolete001.obj
 0002:000021f0       ??_C@_0CJ@MFPGLLFH@nsk?1jvmti?1IsMethodObsolete?1isob@ 00000001800081f0     libisobsolete001.obj
 0002:00002220       ??_C@_0BI@ENEOJHP@Find?5debugee?5class?3?5?$CFs?6@ 0000000180008220     libisobsolete001.obj
 0002:00002238       ??_C@_0DP@MFMMLPOM@?$CIdebugeeClass?5?$DN?5jni?9?$DOFindClass?$CI@ 0000000180008238     libisobsolete001.obj
 0002:00002278       ??_C@_0BH@IDHNHJKP@?5?5?4?4?4?5found?5class?3?5?$CFp?6@ 0000000180008278     libisobsolete001.obj
 0002:00002290       ??_C@_0P@FAMEABDJ@classfileBytes@ 0000000180008290     libisobsolete001.obj
 0002:000022a0       ??_C@_0BH@PMPIFENK@Find?5static?5field?3?5?$CFs?6@ 00000001800082a0     libisobsolete001.obj
 0002:000022c0       ??_C@_0GG@MMDJIFEH@?$CIfieldID?5?$DN?5jni?9?$DOGetStaticFieldI@ 00000001800082c0     libisobsolete001.obj
 0002:00002328       ??_C@_02KCBIMKDL@?$FLB@    0000000180008328     libisobsolete001.obj
 0002:00002330       ??_C@_0BH@CBHPKIDK@?5?5?4?4?4?5got?5fieldID?3?5?$CFp?6@ 0000000180008330     libisobsolete001.obj
 0002:00002348       ??_C@_0DB@LNBEDBAK@Get?5classfile?5bytes?5array?5from?5@ 0000000180008348     libisobsolete001.obj
 0002:00002380       ??_C@_0FD@CEALCFBA@?$CIarray?5?$DN?5?$CIjbyteArray?$CJ?5jni?9?$DOGetS@ 0000000180008380     libisobsolete001.obj
 0002:000023d8       ??_C@_0BM@KDBCJKHI@?5?5?4?4?4?5got?5array?5object?3?5?$CFp?6@ 00000001800083d8     libisobsolete001.obj
 0002:000023f8       ??_C@_0CJ@IMCLCODJ@?$CI?$CKsize?5?$DN?5jni?9?$DOGetArrayLength?$CIar@ 00000001800083f8     libisobsolete001.obj
 0002:00002428       ??_C@_0CA@DFOMIFBE@?5?5?4?4?4?5got?5array?5size?3?5?$CFd?5bytes?6@ 0000000180008428     libisobsolete001.obj
 0002:00002450       ??_C@_0EC@BMGANPNC@?$CIelements?5?$DN?5jni?9?$DOGetByteArrayEl@ 0000000180008450     libisobsolete001.obj
 0002:00002498       ??_C@_0BN@CJGGABDK@?5?5?4?4?4?5got?5elements?5list?3?5?$CFp?6@ 0000000180008498     libisobsolete001.obj
 0002:000024b8       ??_C@_0BO@INNLGEFF@jvmti?9?$DOAllocate?$CI?$CKsize?0?5bytes?$CJ@ 00000001800084b8     libisobsolete001.obj
 0002:000024d8       ??_C@_0BP@DJKEMBMF@?5?5?4?4?4?5created?5bytes?5array?3?5?$CFp?6@ 00000001800084d8     libisobsolete001.obj
 0002:000024f8       ??_C@_0CB@JLCJNBFH@?5?5?4?4?4?5copied?5bytecode?3?5?$CFd?5bytes@ 00000001800084f8     libisobsolete001.obj
 0002:00002520       ??_C@_0BL@MIBLMFCG@Release?5elements?5list?3?5?$CFp?6@ 0000000180008520     libisobsolete001.obj
 0002:00002540       ??_C@_0DK@LPBJCMNH@jni?9?$DOReleaseByteArrayElements?$CIa@ 0000000180008540     libisobsolete001.obj
 0002:00002580       ??_C@_0BA@MKNEJBDK@?5?5?4?4?4?5released?6@ 0000000180008580     libisobsolete001.obj
 0002:00002590       ??_C@_0CA@GPIBFBEH@Wait?5for?5tested?5methods?5to?5run?6@ 0000000180008590     libisobsolete001.obj
 0002:000025b0       ??_C@_0BP@LAIJOMPC@nsk_jvmti_waitForSync?$CItimeout?$CJ@ 00000001800085b0     libisobsolete001.obj
 0002:000025d0       ??_C@_0CO@CNGLMACC@?$DO?$DO?$DO?5Obtain?5bytes?5for?5class?5file@ 00000001800085d0     libisobsolete001.obj
 0002:00002600       ??_C@_0DP@OJABDAOA@getClassfileBytes?$CIjni?0?5jvmti?0?5?$CG@ 0000000180008600     libisobsolete001.obj
 0002:00002640       ??_C@_0CM@KOLNNMJB@?$DO?$DO?$DO?5Find?5tested?5methods?5and?5run@ 0000000180008640     libisobsolete001.obj
 0002:00002670       ??_C@_0CK@OIMDCJJI@nsk?1jvmti?1IsMethodObsolete?1isob@ 0000000180008670     libisobsolete001.obj
 0002:000026a0       ??_C@_0BH@HGFADHMF@Find?5tested?5class?3?5?$CFs?6@ 00000001800086a0     libisobsolete001.obj
 0002:000026b8       ??_C@_0DN@PIMOJJGL@?$CItestedClass?5?$DN?5jni?9?$DOFindClass?$CIT@ 00000001800086b8     libisobsolete001.obj
 0002:000026f8       ??_C@_0CM@PCBLBIAC@Make?5global?5reference?5for?5class@ 00000001800086f8     libisobsolete001.obj
 0002:00002730       ??_C@_0ED@GELBJCOL@?$CItestedClass?5?$DN?5?$CIjclass?$CJ?5jni?9?$DONe@ 0000000180008730     libisobsolete001.obj
 0002:00002778       ??_C@_0BJ@PNFHPOGN@?5?5?4?4?4?5got?5reference?3?5?$CFp?6@ 0000000180008778     libisobsolete001.obj
 0002:00002798       ??_C@_0BJ@OGHGDKAH@Get?5static?5methodID?3?5?$CFs?6@ 0000000180008798     libisobsolete001.obj
 0002:000027c0       ??_C@_0GJ@NAAPBGBL@?$CIstaticMethodID?5?$DN?5jni?9?$DOGetStati@ 00000001800087c0     libisobsolete001.obj
 0002:00002830       ??_C@_0DA@JPABPEJ@?$CIILnsk?1jvmti?1IsMethodObsolete?1i@ 0000000180008830     libisobsolete001.obj
 0002:00002860       ??_C@_0BI@KNDAICKI@?5?5?4?4?4?5got?5methodID?3?5?$CFp?6@ 0000000180008860     libisobsolete001.obj
 0002:00002878       ??_C@_0BL@DGJLEMBP@Get?5instance?5methodID?3?5?$CFs?6@ 0000000180008878     libisobsolete001.obj
 0002:000028a0       ??_C@_0GJ@IHBENABK@?$CIinstanceMethodID?5?$DN?5jni?9?$DOGetMet@ 00000001800088a0     libisobsolete001.obj
 0002:00002910       ??_C@_0N@BEFDDEHE@testedThread@ 0000000180008910     libisobsolete001.obj
 0002:00002920       ??_C@_0CO@FIKGLNEM@Find?5thread?5with?5running?5method@ 0000000180008920     libisobsolete001.obj
 0002:00002950       ??_C@_0EH@KBGOCIDN@?$CItestedThread?5?$DN?5nsk_jvmti_threa@ 0000000180008950     libisobsolete001.obj
 0002:00002998       ??_C@_0CA@IPGOBOEH@?5?5?4?4?4?5got?5thread?5reference?3?5?$CFp?6@ 0000000180008998     libisobsolete001.obj
 0002:000029c0       ??_C@_0EL@HBNCMCJI@?$DO?$DO?$DO?5Testcase?5?$CD1?3?5check?5IsObsole@ 00000001800089c0     libisobsolete001.obj
 0002:00002a10       ??_C@_0BC@BBFONNMK@not?5yet?5redefined@ 0000000180008a10     libisobsolete001.obj
 0002:00002a30       ??_C@_0FE@OLNBGHPF@?$DO?$DO?$DO?5Testcase?5?$CD2?3?5check?5IsObsole@ 0000000180008a30     libisobsolete001.obj
 0002:00002a88       ??_C@_0DD@OJMHEANF@?$DO?$DO?$DO?5Redefine?5class?5while?5method@ 0000000180008a88     libisobsolete001.obj
 0002:00002ac0       ??_C@_0FE@KDMDKKME@redefineClass?$CIjvmti?0?5testedClas@ 0000000180008ac0     libisobsolete001.obj
 0002:00002b20       ??_C@_0EK@OCHJMEOJ@?$DO?$DO?$DO?5Testcase?5?$CD3?3?5check?5IsObsole@ 0000000180008b20     libisobsolete001.obj
 0002:00002b70       ??_C@_09KLOJBFOH@redefined@ 0000000180008b70     libisobsolete001.obj
 0002:00002b80       ??_C@_0FN@NMEFBFBC@?$DO?$DO?$DO?5Testcase?5?$CD4?3?5check?5IsObsole@ 0000000180008b80     libisobsolete001.obj
 0002:00002be0       ??_C@_0BF@MNKEFEOE@?$DO?$DO?$DO?5Clean?5used?5data?6@ 0000000180008be0     libisobsolete001.obj
 0002:00002bf8       ??_C@_0CG@NJNCHHBA@Deallocate?5classfile?5bytes?5arra@ 0000000180008bf8     libisobsolete001.obj
 0002:00002c20       ??_C@_0CC@HHJEOPKH@jvmti?9?$DODeallocate?$CIclassfileByte@ 0000000180008c20     libisobsolete001.obj
 0002:00002c48       ??_C@_0CG@GPPBGHJH@Delete?5global?5eference?5to?5threa@ 0000000180008c48     libisobsolete001.obj
 0002:00002c70       ??_C@_0CD@JEIIOPBJ@jni?9?$DODeleteGlobalRef?$CItestedThre@ 0000000180008c70     libisobsolete001.obj
 0002:00002c98       ??_C@_0CG@LEHDLKLJ@Delete?5global?5reference?5to?5clas@ 0000000180008c98     libisobsolete001.obj
 0002:00002cc0       ??_C@_0CC@JPMJEGPE@jni?9?$DODeleteGlobalRef?$CItestedClas@ 0000000180008cc0     libisobsolete001.obj
 0002:00002ce8       ??_C@_0BH@HPEOJMHL@Let?5debugee?5to?5finish?6@ 0000000180008ce8     libisobsolete001.obj
 0002:00002d00       ??_C@_0BH@LECMGIIA@nsk_jvmti_resumeSync?$CI?$CJ@ 0000000180008d00     libisobsolete001.obj
 0002:00002d18       ??_C@_0CA@MNKGCBCG@nsk_jvmti_parseOptions?$CIoptions?$CJ@ 0000000180008d18     libisobsolete001.obj
 0002:00002d38       ??_C@_0DN@MIAMNFPH@?$CIjvmti?5?$DN?5nsk_jvmti_createJVMTIE@ 0000000180008d38     libisobsolete001.obj
 0002:00002d78       ??_C@_0BO@DBKDIPGD@jvmti?9?$DOAddCapabilities?$CI?$CGcaps?$CJ@ 0000000180008d78     libisobsolete001.obj
 0002:00002d98       ??_C@_0CL@PIACJIPK@nsk_jvmti_setAgentProc?$CIagentPro@ 0000000180008d98     libisobsolete001.obj
 0002:00002de0       ??_C@_1EC@JIJBPKFM@?$AAa?$AAp?$AAi?$AA?9?$AAm?$AAs?$AA?9?$AAw?$AAi?$AAn?$AA?9?$AAc?$AAo?$AAr?$AAe@ 0000000180008de0     MSVCRT:thread_safe_statics.obj
 0002:00002e28       ??_C@_1BK@MGMFAEKH@?$AAk?$AAe?$AAr?$AAn?$AAe?$AAl?$AA3?$AA2?$AA?4?$AAd?$AAl?$AAl@ 0000000180008e28     MSVCRT:thread_safe_statics.obj
 0002:00002e48       ??_C@_0BJ@JEBJOJFJ@SleepConditionVariableCS@ 0000000180008e48     MSVCRT:thread_safe_statics.obj
 0002:00002e68       ??_C@_0BJ@PGPPEPCC@WakeAllConditionVariable@ 0000000180008e68     MSVCRT:thread_safe_statics.obj
 0002:00002e88       _pDefaultRawDllMain        0000000180008e88     MSVCRT:dll_dllmain.obj
 0002:00002e88       _pRawDllMain               0000000180008e88     MSVCRT:dll_dllmain.obj
 0002:00002e90       __xmm@ffffffffffffffffffffffffffffffff 0000000180008e90     MSVCRT:utility.obj
 0002:00002ea0       _load_config_used          0000000180008ea0     MSVCRT:loadcfg.obj
 0002:00003080       _tls_used                  0000000180009080     MSVCRT:tlssup.obj
 0002:000030a8       __volatile_metadata        00000001800090a8     <linker-defined>
 0002:00003480       __rtc_iaa                  0000000180009480     MSVCRT:initsect.obj
 0002:00003488       __rtc_izz                  0000000180009488     MSVCRT:initsect.obj
 0002:00003490       __rtc_taa                  0000000180009490     MSVCRT:initsect.obj
 0002:00003498       __rtc_tzz                  0000000180009498     MSVCRT:initsect.obj
 0002:000034a0       _tls_start                 00000001800094a0     MSVCRT:tlssup.obj
 0002:000034a4       _Init_thread_epoch         00000001800094a4     MSVCRT:thread_safe_statics.obj
 0002:000034a8       _tls_end                   00000001800094a8     MSVCRT:tlssup.obj
 0002:00003bd8       __IMPORT_DESCRIPTOR_KERNEL32 0000000180009bd8     kernel32:KERNEL32.dll
 0002:00003bec       __IMPORT_DESCRIPTOR_VCRUNTIME140 0000000180009bec     vcruntime:VCRUNTIME140.dll
 0002:00003c00       __IMPORT_DESCRIPTOR_api-ms-win-crt-heap-l1-1-0 0000000180009c00     ucrt:api-ms-win-crt-heap-l1-1-0.dll
 0002:00003c14       __IMPORT_DESCRIPTOR_api-ms-win-crt-runtime-l1-1-0 0000000180009c14     ucrt:api-ms-win-crt-runtime-l1-1-0.dll
 0002:00003c28       __IMPORT_DESCRIPTOR_api-ms-win-crt-convert-l1-1-0 0000000180009c28     ucrt:api-ms-win-crt-convert-l1-1-0.dll
 0002:00003c3c       __IMPORT_DESCRIPTOR_api-ms-win-crt-stdio-l1-1-0 0000000180009c3c     ucrt:api-ms-win-crt-stdio-l1-1-0.dll
 0002:00003c50       __IMPORT_DESCRIPTOR_api-ms-win-crt-string-l1-1-0 0000000180009c50     ucrt:api-ms-win-crt-string-l1-1-0.dll
 0002:00003c64       __NULL_IMPORT_DESCRIPTOR   0000000180009c64     kernel32:KERNEL32.dll
 0003:00000030       _Init_global_epoch         000000018000b030     MSVCRT:thread_safe_statics.obj
 0003:00000040       __security_cookie          000000018000b040     MSVCRT:gs_cookie.obj
 0003:00000048       __security_cookie_complement 000000018000b048     MSVCRT:gs_cookie.obj
 0003:00000050       __scrt_native_dllmain_reason 000000018000b050     MSVCRT:utility.obj
 0003:00000058       __isa_available            000000018000b058     MSVCRT:cpu_disp.obj
 0003:0000005c       __isa_enabled              000000018000b05c     MSVCRT:cpu_disp.obj
 0003:00000060       __memset_fast_string_threshold 000000018000b060     MSVCRT:cpu_disp.obj
 0003:00000068       __memset_nt_threshold      000000018000b068     MSVCRT:cpu_disp.obj
 0003:00000070       __scrt_ucrt_dll_is_in_use  000000018000b070     MSVCRT:ucrt_stubs.obj
 0003:00000080       g_wrongHeapCallbacks       000000018000b080     libisobsolete001.obj
 0003:00000100       g_szTagInfo                000000018000b100     libisobsolete001.obj
 0003:00002040       g_tagFlags                 000000018000d040     libisobsolete001.obj
 0003:00002428       g_refsToVerifyCnt          000000018000d428     libisobsolete001.obj
 0003:0000242c       g_fakeUserData             000000018000d42c     libisobsolete001.obj
 0003:00002430       g_tagVisitCount            000000018000d430     libisobsolete001.obj
 0003:000033d0       g_refsToVerify             000000018000e3d0     libisobsolete001.obj
 0003:0001aad0       g_userDataError            0000000180025ad0     libisobsolete001.obj
 0003:0001ac70       ?_OptionsStorage@?1??__local_stdio_printf_options@@9@4_KA 0000000180025c70     libisobsolete001.obj
 0003:0001b238       _tls_index                 0000000180026238     MSVCRT:tlssup.obj
 0003:0001b240       __scrt_current_native_startup_state 0000000180026240     MSVCRT:utility.obj
 0003:0001b248       __scrt_native_startup_lock 0000000180026248     MSVCRT:utility.obj
 0003:0001b288       __scrt_debugger_hook_flag  0000000180026288     MSVCRT:utility_desktop.obj
 0003:0001b290       ?__type_info_root_node@@3U__type_info_node@@A 0000000180026290     MSVCRT:tncleanup.obj
 0003:0001b2a0       ?_OptionsStorage@?1??__local_stdio_scanf_options@@9@4_KA 00000001800262a0     MSVCRT:default_local_stdio_options.obj
 0003:0001b2a8       __favor                    00000001800262a8     MSVCRT:cpu_disp.obj
 0003:0001b2b0       __dyn_tls_init_callback    00000001800262b0     <common>

 entry point at        0001:00003fd0

 Static symbols

 0000:fffd7000       .debug$S                   0000000180000000     isobsolete001.exp
 0000:fffd7000       .debug$S                   0000000180000000     vcruntime:VCRUNTIME140.dll
 0000:fffd7000       .debug$S                   0000000180000000     vcruntime:VCRUNTIME140.dll
 0000:fffd7000       .debug$S                   0000000180000000     vcruntime:VCRUNTIME140.dll
 0000:fffd7000       .debug$S                   0000000180000000     vcruntime:VCRUNTIME140.dll
 0000:fffd7000       .debug$S                   0000000180000000     vcruntime:VCRUNTIME140.dll
 0000:fffd7000       .debug$S                   0000000180000000     vcruntime:VCRUNTIME140.dll
 0000:fffd7000       .debug$S                   0000000180000000     vcruntime:VCRUNTIME140.dll
 0000:fffd7000       .debug$S                   0000000180000000     ucrt:api-ms-win-crt-convert-l1-1-0.dll
 0000:fffd7000       .debug$S                   0000000180000000     ucrt:api-ms-win-crt-heap-l1-1-0.dll
 0000:fffd7000       .debug$S                   0000000180000000     ucrt:api-ms-win-crt-heap-l1-1-0.dll
 0000:fffd7000       .debug$S                   0000000180000000     ucrt:api-ms-win-crt-heap-l1-1-0.dll
 0000:fffd7000       .debug$S                   0000000180000000     ucrt:api-ms-win-crt-heap-l1-1-0.dll
 0000:fffd7000       .debug$S                   0000000180000000     ucrt:api-ms-win-crt-runtime-l1-1-0.dll
 0000:fffd7000       .debug$S                   0000000180000000     ucrt:api-ms-win-crt-runtime-l1-1-0.dll
 0000:fffd7000       .debug$S                   0000000180000000     ucrt:api-ms-win-crt-runtime-l1-1-0.dll
 0000:fffd7000       .debug$S                   0000000180000000     ucrt:api-ms-win-crt-runtime-l1-1-0.dll
 0000:fffd7000       .debug$S                   0000000180000000     ucrt:api-ms-win-crt-runtime-l1-1-0.dll
 0000:fffd7000       .debug$S                   0000000180000000     ucrt:api-ms-win-crt-runtime-l1-1-0.dll
 0000:fffd7000       .debug$S                   0000000180000000     ucrt:api-ms-win-crt-runtime-l1-1-0.dll
 0000:fffd7000       .debug$S                   0000000180000000     ucrt:api-ms-win-crt-runtime-l1-1-0.dll
 0000:fffd7000       .debug$S                   0000000180000000     ucrt:api-ms-win-crt-runtime-l1-1-0.dll
 0000:fffd7000       .debug$S                   0000000180000000     ucrt:api-ms-win-crt-runtime-l1-1-0.dll
 0000:fffd7000       .debug$S                   0000000180000000     ucrt:api-ms-win-crt-runtime-l1-1-0.dll
 0000:fffd7000       .debug$S                   0000000180000000     ucrt:api-ms-win-crt-runtime-l1-1-0.dll
 0000:fffd7000       .debug$S                   0000000180000000     ucrt:api-ms-win-crt-runtime-l1-1-0.dll
 0000:fffd7000       .debug$S                   0000000180000000     ucrt:api-ms-win-crt-runtime-l1-1-0.dll
 0000:fffd7000       .debug$S                   0000000180000000     ucrt:api-ms-win-crt-runtime-l1-1-0.dll
 0000:fffd7000       .debug$S                   0000000180000000     ucrt:api-ms-win-crt-runtime-l1-1-0.dll
 0000:fffd7000       .debug$S                   0000000180000000     ucrt:api-ms-win-crt-stdio-l1-1-0.dll
 0000:fffd7000       .debug$S                   0000000180000000     ucrt:api-ms-win-crt-stdio-l1-1-0.dll
 0000:fffd7000       .debug$S                   0000000180000000     ucrt:api-ms-win-crt-stdio-l1-1-0.dll
 0000:fffd7000       .debug$S                   0000000180000000     ucrt:api-ms-win-crt-stdio-l1-1-0.dll
 0000:fffd7000       .debug$S                   0000000180000000     ucrt:api-ms-win-crt-stdio-l1-1-0.dll
 0000:fffd7000       .debug$S                   0000000180000000     ucrt:api-ms-win-crt-stdio-l1-1-0.dll
 0000:fffd7000       .debug$S                   0000000180000000     ucrt:api-ms-win-crt-stdio-l1-1-0.dll
 0000:fffd7000       .debug$S                   0000000180000000     ucrt:api-ms-win-crt-stdio-l1-1-0.dll
 0000:fffd7000       .debug$S                   0000000180000000     ucrt:api-ms-win-crt-stdio-l1-1-0.dll
 0000:fffd7000       .debug$S                   0000000180000000     ucrt:api-ms-win-crt-stdio-l1-1-0.dll
 0000:fffd7000       .debug$S                   0000000180000000     ucrt:api-ms-win-crt-string-l1-1-0.dll
 0000:fffd7000       .debug$S                   0000000180000000     ucrt:api-ms-win-crt-string-l1-1-0.dll
 0000:fffd7000       .debug$S                   0000000180000000     ucrt:api-ms-win-crt-string-l1-1-0.dll
 0000:fffd7000       .debug$S                   0000000180000000     ucrt:api-ms-win-crt-string-l1-1-0.dll
 0000:fffd7000       .debug$S                   0000000180000000     ucrt:api-ms-win-crt-string-l1-1-0.dll
 0000:fffd7000       .debug$S                   0000000180000000     ucrt:api-ms-win-crt-string-l1-1-0.dll
 0000:fffd7000       .debug$S                   0000000180000000     ucrt:api-ms-win-crt-string-l1-1-0.dll
 0000:fffd7000       .debug$S                   0000000180000000     ucrt:api-ms-win-crt-string-l1-1-0.dll
 0000:fffd7000       .debug$S                   0000000180000000     kernel32:KERNEL32.dll
 0000:fffd7000       .debug$S                   0000000180000000     kernel32:KERNEL32.dll
 0000:fffd7000       .debug$S                   0000000180000000     kernel32:KERNEL32.dll
 0000:fffd7000       .debug$S                   0000000180000000     kernel32:KERNEL32.dll
 0000:fffd7000       .debug$S                   0000000180000000     kernel32:KERNEL32.dll
 0000:fffd7000       .debug$S                   0000000180000000     kernel32:KERNEL32.dll
 0000:fffd7000       .debug$S                   0000000180000000     kernel32:KERNEL32.dll
 0000:fffd7000       .debug$S                   0000000180000000     kernel32:KERNEL32.dll
 0000:fffd7000       .debug$S                   0000000180000000     kernel32:KERNEL32.dll
 0000:fffd7000       .debug$S                   0000000180000000     kernel32:KERNEL32.dll
 0000:fffd7000       .debug$S                   0000000180000000     kernel32:KERNEL32.dll
 0000:fffd7000       .debug$S                   0000000180000000     kernel32:KERNEL32.dll
 0000:fffd7000       .debug$S                   0000000180000000     kernel32:KERNEL32.dll
 0000:fffd7000       .debug$S                   0000000180000000     kernel32:KERNEL32.dll
 0000:fffd7000       .debug$S                   0000000180000000     kernel32:KERNEL32.dll
 0000:fffd7000       .debug$S                   0000000180000000     kernel32:KERNEL32.dll
 0000:fffd7000       .debug$S                   0000000180000000     kernel32:KERNEL32.dll
 0000:fffd7000       .debug$S                   0000000180000000     kernel32:KERNEL32.dll
 0000:fffd7000       .debug$S                   0000000180000000     kernel32:KERNEL32.dll
 0000:fffd7000       .debug$S                   0000000180000000     kernel32:KERNEL32.dll
 0000:fffd7000       .debug$S                   0000000180000000     kernel32:KERNEL32.dll
 0000:fffd7000       .debug$S                   0000000180000000     kernel32:KERNEL32.dll
 0000:fffd7000       .debug$S                   0000000180000000     kernel32:KERNEL32.dll
 0000:fffd7000       .debug$S                   0000000180000000     kernel32:KERNEL32.dll
 0000:fffd7000       .debug$S                   0000000180000000     kernel32:KERNEL32.dll
 0000:fffd7000       .debug$S                   0000000180000000     kernel32:KERNEL32.dll
 0000:fffd7000       .debug$S                   0000000180000000     kernel32:KERNEL32.dll
 0000:fffd7000       .debug$S                   0000000180000000     kernel32:KERNEL32.dll
 0001:00000e4c       addRefToVerify             0000000180001e4c f   libisobsolete001.obj
 0001:00000eb8       agentProc                  0000000180001eb8 f   libisobsolete001.obj
 0001:00001660       agentThreadWrapper         0000000180002660 f   libisobsolete001.obj
 0001:000017cc       checkMethodObsolete        00000001800027cc f   libisobsolete001.obj
 0001:000018fc       checkStackMethodsObsolete  00000001800028fc f   libisobsolete001.obj
 0001:00001d88       check_option               0000000180002d88 f   libisobsolete001.obj
 0001:00001fd0       file_basename              0000000180002fd0 f   libisobsolete001.obj
 0001:00002044       getClassfileBytes          0000000180003044 f   libisobsolete001.obj
 0001:000033b0       redefineClass              00000001800043b0 f   libisobsolete001.obj
 0001:000034ac       startAgentThreadWrapper    00000001800044ac f   libisobsolete001.obj
 0001:000037ec       syncDebuggeeStatus         00000001800047ec f   libisobsolete001.obj
 0001:00003a8c       capture_previous_context   0000000180004a8c f   MSVCRT:gs_report.obj
 0001:00003b00       ?__scrt_initialize_thread_safe_statics@@YAHXZ 0000000180004b00 f   MSVCRT:thread_safe_statics.obj
 0001:00003bd0       ?__scrt_uninitialize_thread_safe_statics@@YAXXZ 0000000180004bd0 f   MSVCRT:thread_safe_statics.obj
 0001:00003c80       $$000000                   0000000180004c80     MSVCRT:amdsecgs.obj
 0001:00003cb0       ?dllmain_crt_dispatch@@YAHQEAUHINSTANCE__@@KQEAX@Z 0000000180004cb0 f   MSVCRT:dll_dllmain.obj
 0001:00003d00       ?dllmain_crt_process_attach@@YAHQEAUHINSTANCE__@@QEAX@Z 0000000180004d00 f   MSVCRT:dll_dllmain.obj
 0001:00003e18       ?dllmain_crt_process_detach@@YAH_N@Z 0000000180004e18 f   MSVCRT:dll_dllmain.obj
 0001:00003e9c       ?dllmain_dispatch@@YAHQEAUHINSTANCE__@@KQEAX@Z 0000000180004e9c f   MSVCRT:dll_dllmain.obj
 0001:000048b0       $$000000                   00000001800058b0     MSVCRT:guard_dispatch.obj
 0001:000048d0       $$000000                   00000001800058d0     MSVCRT:guard_xfg_dispatch.obj
 0001:000048e6       ?fin$0@?0??dllmain_crt_process_attach@@YAHQEAUHINSTANCE__@@QEAX@Z@4HA 00000001800058e6 f   MSVCRT:dll_dllmain.obj
 0001:000048fd       ?fin$0@?0??dllmain_crt_process_detach@@YAH_N@Z@4HA 00000001800058fd f   MSVCRT:dll_dllmain.obj
 0001:00004916       ?fin$1@?0??dllmain_crt_process_detach@@YAH_N@Z@4HA 0000000180005916 f   MSVCRT:dll_dllmain.obj
 0001:0000492a       ?filt$0@?0??dllmain_dispatch@@YAHQEAUHINSTANCE__@@KQEAX@Z@4HA 000000018000592a f   MSVCRT:dll_dllmain.obj
 0001:00004960       __scrt_is_nonwritable_in_current_image$filt$0 0000000180005960 f   MSVCRT:utility.obj
 0002:00000218       ?__scrt_initialize_tss_var@@3P6AHXZEA 0000000180006218     MSVCRT:thread_safe_statics.obj
 0002:00000340       ?opcLengths@@3QBEB         0000000180006340     libisobsolete001.obj
 0002:00002dc8       GS_ExceptionPointers       0000000180008dc8     MSVCRT:gs_report.obj
 0002:000034b0       $unwind$fprintf            00000001800094b0     libisobsolete001.obj
 0002:000034bc       $unwind$printf             00000001800094bc     libisobsolete001.obj
 0002:000034c8       $unwind$?NewObject@JNIEnv_@@QEAAPEAV_jobject@@PEAV_jclass@@PEAU_jmethodID@@ZZ 00000001800094c8     libisobsolete001.obj
 0002:000034c8       $unwind$nsk_lcomplain      00000001800094c8     libisobsolete001.obj
 0002:000034c8       $unwind$nsk_ldisplay       00000001800094c8     libisobsolete001.obj
 0002:000034d0       $unwind$nsk_jvmti_waitForSync 00000001800094d0     libisobsolete001.obj
 0002:000034d0       $unwind$nsk_lvdisplay      00000001800094d0     libisobsolete001.obj
 0002:000034d0       $unwind$_RTC_Initialize    00000001800094d0     MSVCRT:initsect.obj
 0002:000034d0       $unwind$_RTC_Terminate     00000001800094d0     MSVCRT:initsect.obj
 0002:000034d0       $unwind$?__scrt_initialize_thread_safe_statics@@YAHXZ 00000001800094d0     MSVCRT:thread_safe_statics.obj
 0002:000034dc       $unwind$nsk_complain       00000001800094dc     libisobsolete001.obj
 0002:000034dc       $unwind$nsk_printf         00000001800094dc     libisobsolete001.obj
 0002:000034e4       $unwind$nsk_lvcomplain     00000001800094e4     libisobsolete001.obj
 0002:000034fc       $unwind$nsk_ltrace         00000001800094fc     libisobsolete001.obj
 0002:000034fc       $unwind$__report_gsfailure 00000001800094fc     MSVCRT:gs_report.obj
 0002:00003504       $unwind$nsk_lvtrace        0000000180009504     libisobsolete001.obj
 0002:00003504       $unwind$__raise_securityfailure 0000000180009504     MSVCRT:gs_report.obj
 0002:00003504       $unwind$__scrt_initialize_crt 0000000180009504     MSVCRT:utility.obj
 0002:00003504       $unwind$__scrt_initialize_onexit_tables 0000000180009504     MSVCRT:utility.obj
 0002:00003504       $unwind$__scrt_release_startup_lock 0000000180009504     MSVCRT:utility.obj
 0002:00003504       $unwind$__scrt_uninitialize_crt 0000000180009504     MSVCRT:utility.obj
 0002:00003504       $unwind$_onexit            0000000180009504     MSVCRT:utility.obj
 0002:0000350c       $unwind$nsk_lverify        000000018000950c     libisobsolete001.obj
 0002:0000351c       $unwind$nsk_vprintf        000000018000951c     libisobsolete001.obj
 0002:0000352c       $unwind$?nsk_jni_lverify@@YAHHPEAUJNIEnv_@@HQEBDH1ZZ 000000018000952c     libisobsolete001.obj
 0002:00003540       $unwind$?nsk_jni_check_exception@@YAHPEAUJNIEnv_@@QEBDH@Z 0000000180009540     libisobsolete001.obj
 0002:0000355c       $unwind$nsk_jvmti_parseOptions 000000018000955c     libisobsolete001.obj
 0002:00003578       $unwind$nsk_jvmti_createJVMTIEnv 0000000180009578     libisobsolete001.obj
 0002:0000358c       $unwind$Java_nsk_jvmti_unit_FollowReferences_FollowRefObjects_resetTags 000000018000958c     libisobsolete001.obj
 0002:0000358c       $unwind$addRefToVerify     000000018000958c     libisobsolete001.obj
 0002:0000358c       $unwind$nsk_jvmti_resetAgentData 000000018000958c     libisobsolete001.obj
 0002:0000358c       $unwind$nsk_jvmti_resumeSync 000000018000958c     libisobsolete001.obj
 0002:0000358c       $unwind$nsk_jvmti_setFailStatus 000000018000958c     libisobsolete001.obj
 0002:0000358c       $unwind$__scrt_initialize_default_local_stdio_options 000000018000958c     MSVCRT:default_local_stdio_options.obj
 0002:0000358c       $unwind$?dllmain_crt_dispatch@@YAHQEAUHINSTANCE__@@KQEAX@Z 000000018000958c     MSVCRT:dll_dllmain.obj
 0002:0000358c       $unwind$DllMain            000000018000958c     MSVCRT:dll_dllmain_stub.obj
 0002:0000358c       $unwind$__GSHandlerCheck   000000018000958c     MSVCRT:gshandler.obj
 0002:0000358c       $unwind$?__scrt_uninitialize_thread_safe_statics@@YAXXZ 000000018000958c     MSVCRT:thread_safe_statics.obj
 0002:0000358c       $unwind$__scrt_acquire_startup_lock 000000018000958c     MSVCRT:utility.obj
 0002:0000358c       $unwind$__scrt_dllmain_after_initialize_c 000000018000958c     MSVCRT:utility.obj
 0002:0000358c       $unwind$__scrt_dllmain_before_initialize_c 000000018000958c     MSVCRT:utility.obj
 0002:0000358c       $unwind$__scrt_dllmain_crt_thread_attach 000000018000958c     MSVCRT:utility.obj
 0002:0000358c       $unwind$__scrt_dllmain_crt_thread_detach 000000018000958c     MSVCRT:utility.obj
 0002:0000358c       $unwind$__scrt_dllmain_uninitialize_c 000000018000958c     MSVCRT:utility.obj
 0002:0000358c       $unwind$__scrt_dllmain_uninitialize_critical 000000018000958c     MSVCRT:utility.obj
 0002:0000358c       $unwind$atexit             000000018000958c     MSVCRT:utility.obj
 0002:00003594       $unwind$nsk_jvmti_threadByName 0000000180009594     libisobsolete001.obj
 0002:000035ac       $unwind$nsk_jvmti_lverify  00000001800095ac     libisobsolete001.obj
 0002:000035c0       $unwind$exitOnError        00000001800095c0     libisobsolete001.obj
 0002:000035d0       $unwind$check_option       00000001800095d0     libisobsolete001.obj
 0002:000035d0       $unwind$_DllMainCRTStartup 00000001800095d0     MSVCRT:dll_dllmain.obj
 0002:000035e0       $unwind$Java_nsk_share_jvmti_ArgumentHandler_getAgentOptionsString 00000001800095e0     libisobsolete001.obj
 0002:000035f4       $unwind$Java_nsk_jvmti_unit_FollowReferences_FollowRefObjects_getTag 00000001800095f4     libisobsolete001.obj
 0002:000035f4       $unwind$Java_nsk_share_jvmti_DebugeeClass_checkStatus 00000001800095f4     libisobsolete001.obj
 0002:000035f4       $unwind$agentThreadWrapper 00000001800095f4     libisobsolete001.obj
 0002:00003604       $unwind$startAgentThreadWrapper 0000000180009604     libisobsolete001.obj
 0002:00003620       $unwind$syncDebuggeeStatus 0000000180009620     libisobsolete001.obj
 0002:00003620       $unwind$__scrt_dllmain_exception_filter 0000000180009620     MSVCRT:utility.obj
 0002:00003634       $unwind$Java_nsk_share_jvmti_DebugeeClass_resetAgentData 0000000180009634     libisobsolete001.obj
 0002:0000363c       $unwind$MA_checkStatus     000000018000963c     libisobsolete001.obj
 0002:00003650       $unwind$Java_nsk_jvmti_unit_FollowReferences_FollowRefObjects_setTag 0000000180009650     libisobsolete001.obj
 0002:00003668       $unwind$Java_nsk_jvmti_unit_FollowReferences_FollowRefObjects_addRefToVerify 0000000180009668     libisobsolete001.obj
 0002:00003684       $unwind$Agent_Initialize   0000000180009684     libisobsolete001.obj
 0002:000036a0       $unwind$checkMethodObsolete 00000001800096a0     libisobsolete001.obj
 0002:000036b8       $unwind$checkStackMethodsObsolete 00000001800096b8     libisobsolete001.obj
 0002:000036dc       $unwind$redefineClass      00000001800096dc     libisobsolete001.obj
 0002:000036f0       $unwind$getClassfileBytes  00000001800096f0     libisobsolete001.obj
 0002:0000370c       $unwind$agentProc          000000018000970c     libisobsolete001.obj
 0002:00003728       $unwind$capture_previous_context 0000000180009728     MSVCRT:gs_report.obj
 0002:00003734       $unwind$__GSHandlerCheckCommon 0000000180009734     MSVCRT:gshandler.obj
 0002:00003740       $xdatasym                  0000000180009740     MSVCRT:amdsecgs.obj
 0002:00003744       $unwind$?dllmain_crt_process_attach@@YAHQEAUHINSTANCE__@@QEAX@Z 0000000180009744     MSVCRT:dll_dllmain.obj
 0002:00003780       $unwind$?fin$0@?0??dllmain_crt_process_attach@@YAHQEAUHINSTANCE__@@QEAX@Z@4HA 0000000180009780     MSVCRT:dll_dllmain.obj
 0002:00003780       $unwind$?fin$0@?0??dllmain_crt_process_detach@@YAH_N@Z@4HA 0000000180009780     MSVCRT:dll_dllmain.obj
 0002:00003780       $unwind$?fin$1@?0??dllmain_crt_process_detach@@YAH_N@Z@4HA 0000000180009780     MSVCRT:dll_dllmain.obj
 0002:00003788       $unwind$?dllmain_crt_process_detach@@YAH_N@Z 0000000180009788     MSVCRT:dll_dllmain.obj
 0002:000037dc       $unwind$?dllmain_dispatch@@YAHQEAUHINSTANCE__@@KQEAX@Z 00000001800097dc     MSVCRT:dll_dllmain.obj
 0002:00003804       $unwind$?filt$0@?0??dllmain_dispatch@@YAHQEAUHINSTANCE__@@KQEAX@Z@4HA 0000000180009804     MSVCRT:dll_dllmain.obj
 0002:0000380c       $unwind$__scrt_is_nonwritable_in_current_image 000000018000980c     MSVCRT:utility.obj
 0002:0000382c       $unwind$__scrt_is_nonwritable_in_current_image$filt$0 000000018000982c     MSVCRT:utility.obj
 0002:00003834       $unwind$__scrt_fastfail    0000000180009834     MSVCRT:utility_desktop.obj
 0002:00003844       $unwind$__security_init_cookie 0000000180009844     MSVCRT:gs_support.obj
 0002:00003850       $unwind$__isa_available_init 0000000180009850     MSVCRT:cpu_disp.obj
 0002:00003860       $xdatasym                  0000000180009860     MSVCRT:guard_dispatch.obj
 0002:00003868       $xdatasym                  0000000180009868     MSVCRT:guard_xfg_dispatch.obj
 0002:00003870       .edata                     0000000180009870     isobsolete001.exp
 0002:00003898       rgpv                       0000000180009898     isobsolete001.exp
 0002:000038d0       rgszName                   00000001800098d0     isobsolete001.exp
 0002:00003908       rgwOrd                     0000000180009908     isobsolete001.exp
 0002:00003924       szName                     0000000180009924     isobsolete001.exp
 0002:00003936       $N00001                    0000000180009936     isobsolete001.exp
 0002:00003945       $N00002                    0000000180009945     isobsolete001.exp
 0002:00003952       $N00003                    0000000180009952     isobsolete001.exp
 0002:00003997       $N00004                    0000000180009997     isobsolete001.exp
 0002:000039d4       $N00005                    00000001800099d4     isobsolete001.exp
 0002:00003a1c       $N00006                    0000000180009a1c     isobsolete001.exp
 0002:00003a5c       $N00007                    0000000180009a5c     isobsolete001.exp
 0002:00003a99       $N00008                    0000000180009a99     isobsolete001.exp
 0002:00003ad4       $N00009                    0000000180009ad4     isobsolete001.exp
 0002:00003b02       $N00010                    0000000180009b02     isobsolete001.exp
 0002:00003b33       $N00011                    0000000180009b33     isobsolete001.exp
 0002:00003b62       $N00012                    0000000180009b62     isobsolete001.exp
 0002:00003b91       $N00013                    0000000180009b91     isobsolete001.exp
 0002:00003bc6       $N00014                    0000000180009bc6     isobsolete001.exp
 0002:0000402a       .idata$6                   000000018000a02a     kernel32:KERNEL32.dll
 0002:0000408e       .idata$6                   000000018000a08e     vcruntime:VCRUNTIME140.dll
 0002:00004220       .idata$6                   000000018000a220     ucrt:api-ms-win-crt-heap-l1-1-0.dll
 0002:00004240       .idata$6                   000000018000a240     ucrt:api-ms-win-crt-runtime-l1-1-0.dll
 0002:00004262       .idata$6                   000000018000a262     ucrt:api-ms-win-crt-convert-l1-1-0.dll
 0002:00004284       .idata$6                   000000018000a284     ucrt:api-ms-win-crt-stdio-l1-1-0.dll
 0002:000042a4       .idata$6                   000000018000a2a4     ucrt:api-ms-win-crt-string-l1-1-0.dll
 0003:00000000       ?codeAttributeName@@3PEBDEB 000000018000b000     libisobsolete001.obj
 0003:00000008       ?lineNumberAttributeName@@3PEBDEB 000000018000b008     libisobsolete001.obj
 0003:00000010       ?localVarAttributeName@@3PEBDEB 000000018000b010     libisobsolete001.obj
 0003:00000018       ?localVarTypeAttributeName@@3PEBDEB 000000018000b018     libisobsolete001.obj
 0003:00000020       ?stackMapAttributeName@@3PEBDEB 000000018000b020     libisobsolete001.obj
 0003:00000028       ?callBytes@@3PAEA          000000018000b028     libisobsolete001.obj
 0003:0000002c       ?allocBytes@@3PAEA         000000018000b02c     libisobsolete001.obj
 0003:0001aad4       redefineAttempted          0000000180025ad4     libisobsolete001.obj
 0003:0001aad8       nsk_context                0000000180025ad8     libisobsolete001.obj
 0003:0001aae4       redefineSucceed            0000000180025ae4     libisobsolete001.obj
 0003:0001aae8       agentFailed                0000000180025ae8     libisobsolete001.obj
 0003:0001aaec       currentAgentStatus         0000000180025aec     libisobsolete001.obj
 0003:0001aaf0       context                    0000000180025af0     libisobsolete001.obj
 0003:0001aba8       agentThread                0000000180025ba8     libisobsolete001.obj
 0003:0001abb0       agentThreadProc            0000000180025bb0     libisobsolete001.obj
 0003:0001abb8       agentThreadArg             0000000180025bb8     libisobsolete001.obj
 0003:0001abc0       agent_data                 0000000180025bc0     libisobsolete001.obj
 0003:0001abd0       jvmti_env                  0000000180025bd0     libisobsolete001.obj
 0003:0001abd8       jvm                        0000000180025bd8     libisobsolete001.obj
 0003:0001abe0       jni_env                    0000000180025be0     libisobsolete001.obj
 0003:0001abe8       checkStatus_func           0000000180025be8     libisobsolete001.obj
 0003:0001abf0       ?codeAttributeIndex@@3GA   0000000180025bf0     libisobsolete001.obj
 0003:0001abf4       ?lineNumberAttributeIndex@@3GA 0000000180025bf4     libisobsolete001.obj
 0003:0001abf8       ?localVarAttributeIndex@@3GA 0000000180025bf8     libisobsolete001.obj
 0003:0001abfc       ?localVarTypeAttributeIndex@@3GA 0000000180025bfc     libisobsolete001.obj
 0003:0001ac00       ?stackMapAttributeIndex@@3GA 0000000180025c00     libisobsolete001.obj
 0003:0001ac04       ?stackFrameOffset@@3GA     0000000180025c04     libisobsolete001.obj
 0003:0001ac08       ?mode@@3HA                 0000000180025c08     libisobsolete001.obj
 0003:0001ac0c       ?constantPoolSize@@3GA     0000000180025c0c     libisobsolete001.obj
 0003:0001ac10       ?orig@@3PEBEEB             0000000180025c10     libisobsolete001.obj
 0003:0001ac18       ?gen@@3PEAEEA              0000000180025c18     libisobsolete001.obj
 0003:0001ac20       ?inputPos@@3PEAEEA         0000000180025c20     libisobsolete001.obj
 0003:0001ac28       ?endPos@@3PEBEEB           0000000180025c28     libisobsolete001.obj
 0003:0001ac30       ?genPos@@3PEAEEA           0000000180025c30     libisobsolete001.obj
 0003:0001ac38       ?markPos@@3PEAEEA          0000000180025c38     libisobsolete001.obj
 0003:0001ac40       ?constantPool@@3PEAPEADEA  0000000180025c40     libisobsolete001.obj
 0003:0001ac48       ?constantPoolCount@@3GA    0000000180025c48     libisobsolete001.obj
 0003:0001ac4c       ?zeroBytes@@3PAEA          0000000180025c4c     libisobsolete001.obj
 0003:0001ac50       ?codeLength@@3IA           0000000180025c50     libisobsolete001.obj
 0003:0001ac58       ?map@@3PEAIEA              0000000180025c58     libisobsolete001.obj
 0003:0001ac60       ?widening@@3PEACEA         0000000180025c60     libisobsolete001.obj
 0003:0001ac68       timeout                    0000000180025c68     libisobsolete001.obj
 0003:0001ac80       GS_ExceptionRecord         0000000180025c80     MSVCRT:gs_report.obj
 0003:0001ad20       GS_ContextRecord           0000000180025d20     MSVCRT:gs_report.obj
 0003:0001b1f0       ?g_tss_cv@@3U_RTL_CONDITION_VARIABLE@@A 00000001800261f0     MSVCRT:thread_safe_statics.obj
 0003:0001b1f8       ?g_tss_event@@3PEAXEA      00000001800261f8     MSVCRT:thread_safe_statics.obj
 0003:0001b200       ?g_tss_mutex@@3U_RTL_CRITICAL_SECTION@@A 0000000180026200     MSVCRT:thread_safe_statics.obj
 0003:0001b228       ?g_sleep_condition_variable_cs@@3P6AHPEAU_RTL_CONDITION_VARIABLE@@PEAU_RTL_CRITICAL_SECTION@@K@ZEA 0000000180026228     MSVCRT:thread_safe_statics.obj
 0003:0001b230       ?g_wake_all_condition_variable@@3P6AXPEAU_RTL_CONDITION_VARIABLE@@@ZEA 0000000180026230     MSVCRT:thread_safe_statics.obj
 0003:0001b23c       ?__proc_attached@@3HA      000000018002623c     MSVCRT:dll_dllmain.obj
 0003:0001b250       ?is_initialized_as_dll@@3_NA 0000000180026250     MSVCRT:utility.obj
 0003:0001b251       ?module_local_atexit_table_initialized@@3_NA 0000000180026251     MSVCRT:utility.obj
 0003:0001b258       ?module_local_atexit_table@@3U_onexit_table_t@@A 0000000180026258     MSVCRT:utility.obj
 0003:0001b270       ?module_local_at_quick_exit_table@@3U_onexit_table_t@@A 0000000180026270     MSVCRT:utility.obj
